:104A1E00534E000006FF507E224E4B4E5144002056
:104A2E0054534E00FE0408FF50B2345242485144D3
:104A3E0000FE09FFFD104C8A8688888688888A8841
:104A4E00868887FE0400FF107E8A88848886888A7E
:104A5E0088868887FE0500FF10B28A888484868C3B
:104A6E00FE0AFF504C204954525344002054534EDA
:104A7E0000FE0406FF507E224E4B4E510020545332
:104A8E004E00FE0509FF50B232404B485100FE0A5F
:104A9E00FFFD104C8C848C848C848C848C848C8450
:104AAE0086868600FF107E8C848C848C848C848C0D
:104ABE00848C8486868600FF10B28C848C8487FE5C
:104ACE000B00FF10618CFF10698CFF10938CFF1090
:104ADE009B8CFF504CB400B500C000C100B600B7AF
:104AEE0000FE0406FF507EB400B500A100A200B681
:104AFE0000B700FE0406FF50B2B200B300FE0C0B6E
:104B0E00FF5061CC0000FF5069CD0000FF5093CCE8
:104B1E000000FF509BCD0000FFFD104C8C848C8458
:104B2E008C848C848C848C8486868600FF107E8C8C
:104B3E00848C848C848C848C848C8486868600FF02
:104B4E0010B28C848C8487FE0B00FF10618CFF10DA
:104B5E00698CFF10938CFF109B8CFF504CB400D5CA
:104B6E0000C000C100D400B700FE0406FF507EB4A2
:104B7E0000D500A100A200D400B700FE0406FF502D
:104B8E00B2DA00DB00FE0C0BFF5061CC0000FF50D0
:104B9E0069CD0000FF5093CC0000FF509BCD00006C
:104BAE00FFFD104C8C848C848C848C848C848C843F
:104BBE0086868600FF107E8C848C848C848C848CFC
:104BCE00848C848C848400FF10B28C848C8487FE49
:104BDE000B00FF10618C8CFF10698C8C8CFF109376
:104BEE008C8CFF109B8C8C8CFF504CB400B500D974
:104BFE0000C100B600B700FE0406FF507EB400B53B
:104C0E0000D600C000CD00B600B7000004FF50B2C1
:104C1E00D700D800FE0C0BFF5061D3D000FF5069B7
:104C2E00D0D0D1FF5093D3D000FF509BD0D0D1FF26
:104C3E00FD104C8A88FE078A8A88FE0500FE14FF46
:104C4E00107E8A8A8A888A848A88888487FE048667
:104C5E000088888800868CFE0C8600FE03FF10B24A
:104C6E008A8A8A888A848A88888487FE048600884D
:104C7E00888800868CFE0C8600FF10E48A8A8A885B
:104C8E0088848A888687FE060088888800868AFE41
:104C9E000C8600FE07FF111C8A8688888488FE0415
:104CAE008688FE050088888800868CFE0C8600FFAC
:104CBE00114E8A8884868CFE0BFF504C00FE0F0C22
:104CCE00FE14FF507E00FE0F04000000040D00FED7
:104CDE000C0CFE04FF50B200FE0F04000000040D89
:104CEE0000FE0C0C0CFF50E400FE0F04000000044C
:104CFE0000002E2D00FE042E25250000000CFE07C0
:104D0E00FF511C00FE0F06000000040D00FE0C0CEF
:104D1E000CFF514E00FE0FFF903C00FE0540FE0AB8
:104D2E000040FE0F00FE1840FE0A0040FE0F00403D
:104D3E0040400040E0FE0C4000FE0740FE0A0040EE
:104D4E00FE0F004040400040E0FE0C4000FE0540DB
:104D5E00FE0A0040FE0F00404040000040FE0C00E6
:104D6E00FE0C40FE0A0040FE0F004040400040E0B6
:104D7E00FE0C4000FE0540FE0A0040FE0F20FE28FD
:104D8E00FFFD104C8A88FE078A8A88FE0500FF10F8
:104D9E007E8A8A8A888A848A88888487FE04860026
:104DAE00FF10B28A8A8A888A848A88888487FE0459
:104DBE008600FF10E48A8A8A8888848A888687FE1D
:104DCE000600FF111C8A868888888488FE048688DF
:104DDE00FE0400FF114E8A8884868CFE0BFF504C19
:104DEE002B404D465440464400FE070CFF507E2E8D
:104DFE00322300270B2F4E520B00FE0504FF50B23C
:104E0E002E322300350B2F4E520B00FE0504FF50A1
:104E1E00E42E32230033484C445100FE0604FF5169
:104E2E001C3351404D524B5442444D5300FE040628
:104E3E00FF514E2457485300FE0BFFFD104C8A883D
:104E4E00868888888788FE0800FF107E8A848A8874
:104E5E008884888A8A8A86FE0500FF10B28A848A30
:104E6E00888884888A8A8A86FE0500FF10E48A88EC
:104E7E00888784878888888486888A8A8A00FF1132
:104E8E001C8A84888886888886888884888884880E
:104E9E0000FF114E8A8888888CFE0BFF504C324FD3
:104EAE00514042474400FE0808FF507E270B2F4E0C
:104EBE00520B002E322300FE0508FF50B2350B2F89
:104ECE004E520B002E322300FE0508FF50E4204DFB
:104EDE005944484644594448530D2E322304FF5139
:104EEE001C2B4842475343545142474B815248462C
:104EFE000EFF514E244D434400FE0BFFFD104C8A15
:104F0E00888888888887FE0900FF107E8A888884B2
:104F1E0086848888888A848A8A8A8800FF10B28A62
:104F2E0088888486848888888A848A8A8A8800FF0A
:104F3E0010E48A8886888888888686848888888807
:104F4E008800FF111C8A86888888848888848888CF
:104F5E0087FE0400FF114E8A8884868688868CFE22
:104F6E0008FF504C2B404D46544400FE0907FF509D
:104F7E007E2F4E524853484E4D00270B2E322300A3
:104F8E0004FF50B22F4E524853484E4D00350B2E53
:104F9E0032230004FF50E42354518544004045451C
:104FAE0048424740464408FF511C3351404D524B36
:104FBE00544248434400FE040CFF514E30544853B3
:104FCE0053445100FE08FFFD104C8A84888888885F
:104FDE008888848888FE0500FF107E8A88878487EB
:104FEE0084888888888A848A8A8A00FF10B28A8890
:104FFE0087848784888888888A848A8A8A00FF10B2
:10500E00E48A888A888888888488888488888888BA
:10501E0000FF111C8A8688888488888488FE070091
:10502E00FF114E8A88888486888AFE0900FF504CBC
:10503E002B484D4654404646484E00FE0508FF504C
:10504E007E2F4E524859484E4D4400270B2E322388
:10505E0004FF50B22F4E524859484E4D4400350B66
:10506E002E322304FF50E433444C4F4E004348523B
:10507E004F4B4058000004FF511C335140524B54CB
:10508E004248434E00FE0508FF514E3452424851ED
:10509E004400FE09FFFD104C8A888888888886881F
:1050AE0087FE0700FF107E8A888884888488888817
:1050BE008A848A8A8A8600FF10B28A8888848884C5
:1050CE008888888A848A8A8A8600FF10E48A84887F
:1050DE008A888888888888888888868400FF111C3A
:1050EE008A868888888488888488FE0600FF114E08
:1050FE008A888484868CFE0AFF504C2B444D46547D
:10510E0040494400FE0707FF507E2F4E524842484A
:10511E008D4D00270B2E32230004FF50B22F4E521E
:10512E004842488D4D00350B2E32230004FF50E4CB
:10513E003348444C4F4E00444D004F404D530B06E8
:10514E00FF511C3351404D524B914248434E00FE8D
:10515E000408FF514E32404B485100FE0AFFFD102D
:10516E004C8C848C848C848C8487FE0700FF107E8C
:10517E008C848C848C848C848C848C84868686002F
:10518E00FF10B28C848C848C848C848C848C84866A
:10519E00868600FF10E48C848C848C848C8487FE3D
:1051AE000700FF111C8C848C848C848C848C8487E7
:1051BE00FE0500FF114E8C848C8487FE0B00FF10C1
:1051CE00FA8CFF11008CFF504CB800B900BA00D316
:1051DE0000FE0807FF507EBA00BB00A800A900AC75
:1051EE0000AD00FE0406FF50B2BA00BB00AA00AB31
:1051FE0000AC00AD00FE0406FF50E4BA00BB00AEEA
:10520E0000C800FE0807FF511CBA00BB00CA00CE42
:10521E0000CF00FE0605FF514EB200B300FE0C0B90
:10522E00FF50FAB30000FF5100C90000FFFD104C03
:10523E008C848C848C848C8487FE0700FF107E8C7B
:10524E00848C848C848C848C848C8486868600FFEB
:10525E0010B28C848C848C848C848C848C84868612
:10526E008600FF10E48C848C848C848C8487FE07EB
:10527E0000FF111C8C848C848C848C848C8487FE1F
:10528E000500FF114E8C848C8487FE0B00FF10FAF4
:10529E008CFF11008CFF504CE200B900D600D700F5
:1052AE00FE0807FF507ED600D800A800A900AC006B
:1052BE00AD00FE0406FF50B2D600D800AA00AB0027
:1052CE00AC00AD00FE0406FF50E4D600D800E000AE
:1052DE00E300FE0807FF511CD600D800CA00CE001E
:1052EE00CF00FE0605FF514EDA00DB00FE0C0BFF71
:1052FE0050FADB0000FF5100E50000FFFD104C8C62
:10530E00848C848C848C8487FE0700FF107E8C84B2
:10531E008C848C848C848C848C848C848400FF108C
:10532E00B28C848C848C848C848C848C848C8484C9
:10533E0000FF10E48C848C848C848C848C848C840C
:10534E008C848400FF111C8C848C848C8487FE09D1
:10535E0000FF114E8C848C8487FE0B00FF10FA8C9C
:10536E00FF11008CFF504CB900B800BA00A000FE2F
:10537E000807FF507EBB00A500CD00A800A900AC19
:10538E0000AD000004FF50B2BB00A500CD00AA0086
:10539E00AB00AC00AD000004FF50E4BB00A500CD97
:1053AE00009F00DD00B300CD000004FF511CCA00B9
:1053BE00CE00CF00FE0A09FF514ED700D800FE0CDA
:1053CE000BFF50FA9B0000FF51009C0000FFFD10E8
:1053DE004C8A8488888884888A88888688FE040017
:1053EE00FE14FF107E8A8A8888888A888488888638
:1053FE0087FE0400888888008688FE0F00FF10B2A2
:10540E008A8888888687FE0A0088888800868A8A25
:10541E008C8AFE098600FF10E48A848A8888848636
:10542E008488FE070088888800868CFE0C8600FE25
:10543E0007FF111C8A8884868888888C8C87FE06D4
:10544E0000FE14FF114E00FE0FFF504C00FE0F0C1D
:10545E00FE14FF507E00FE0F04000000040007053E
:10546E00010E050101000803010E0501010CFF509C
:10547E00B200FE0F0A000000040038243200FE05C0
:10548E002D2E0000000CFF50E400FE0F0A0000005D
:10549E00040D00FE0C0CFE08FF511C00FE0F0CFE4E
:1054AE0014FF514E0CFE0FFF903C00FE0540FE0A0D
:1054BE000040FE0F00FE1840FE0A0040FE0F0040A6
:1054CE0040400040FE08E040FE0700FE0540FE0A98
:1054DE000040FE0F004040400040FE0E00FE054022
:1054EE00FE0A0040FE0F004040400040E0FE0C402F
:1054FE0000FE0B40FE0A0040FE0F00FE1840FE0AA2
:10550E0000FE1020FE28FFFD104C8A8488888884B7
:10551E00888A88888688FE0400FF107E8A8A88889A
:10552E00888A888488888687FE0400FF10B28A885D
:10553E0088888687FE0A00FF10E48A8884888A8815
:10554E0087FE0900FF111C8A88848688FE0B00FFE7
:10555E00114E00FE0FFF504C3248464D404B00326C
:10556E004E5451424400000CFF507E2C4E434400DA
:10557E0032444B44425300FE0404FF50B2314452B5
:10558E00445300FE0A0AFF50E4354E4B544C44007F
:10559E00FE0909FF511C2457485300FE0B04FF510E
:1055AE004E0CFE0FFFFD104C8A84888888848884F8
:1055BE0088FE0700FF107E8A888888888A888884FB
:1055CE0087FE0600FF10B28A8886888888888886BB
:1055DE0088888887FE0300FF10E48A8884888A887A
:1055EE0087FE0900FF111C8A8888888CFE0BFF50ED
:1055FE004C3248464D404B44484D46404D460000C7
:10560E000AFF507E2C4E4354525640474B00FE0626
:10561E0006FF50B239545192424A52445359444DA6
:10562E0000FE0305FF50E4354E4B544C4400FE097A
:10563E0009FF511C244D434400FE0BFFFD104C8A04
:10564E00888686888887FE0900FF107E8A8884886F
:10565E008886848888888A8888888800FF10B28A1D
:10566E00888488848684888484888886888800FFD5
:10567E0010E48A8884888A8887FE0900FF111C8AB4
:10568E008884868688868CFE08FF504C244D5351A4
:10569E00854400FE090BFF507E32854B4442534831
:1056AE004E4D004C4E43440006FF50B23185484DDE
:1056BE00485348404B48524451000016FF50E435C1
:1056CE004E4B544C4400FE0909FF511C30544853B4
:1056DE0053445100FE08FFFD104C8488888688884C
:1056EE00888888FE0600FF107E8A888488888488D1
:1056FE008888888A8888888800FF10B28A88848A79
:10570E00888888868887FE0600FF10E48A88848849
:10571E008A8887FE0900FF111C8A88888486888AF9
:10572E00FE0900FF504C284D46514452524E00FE89
:10573E00060EFF507E32444B4459484E4D44004CA9
:10574E004E434E0004FF50B23144484C4F4E52531C
:10575E004000FE0608FF50E4354E4B544C4400FE0C
:10576E000909FF511C34524248514400FE09FFFD05
:10577E00104C8A88868688888887FE0800FF107EEF
:10578E008A88848888848888888A88888888880017
:10579E00FF10B28A888886888886888687FE0600EB
:1057AE00FF10E48A8884888A888887FE0800FF11A3
:1057BE001C8A888484868CFE0AFF504C244D5351DB
:1057CE0040434000FE080AFF507E32444B44420BD9
:1057DE004344004C4E434E000004FF50B23144404F
:1057EE0049545253405100FE060AFF50E4354E4BC9
:1057FE00544C444D00FE0808FF511C32404B48519A
:10580E0000FE0AFFFD104C8C848C848C848C848763
:10581E00FE0700FF107E8C848C848C848C8487FE23
:10582E000700FF10B28C848C8487FE0B00FF10E4FF
:10583E008C848C8487FE0B00FF111C8C848C8487D7
:10584E00FE0B00FF10C78CFF10CF8CFF504CBC001E
:10585E00BD00BA00D300FE0807FF507EC000C10095
:10586E00BA00D300FE0807FF50B2CB00AD00FE0C0D
:10587E000BFF50E4BE00BF00FE0C0BFF511CB2002C
:10588E00B300FE0C0BFF50C7CC0000FF50CFCD0075
:10589E0000FFFD104C8C848C848C848C8487FE07D6
:1058AE0000FF107E8C848C848C848C8487FE070091
:1058BE00FF10B28C848C8487FE0B00FF10E48C8466
:1058CE008C8487FE0B00FF111C8C848C8487FE0B4E
:1058DE0000FF10C78CFF10CF8CFF504CBC00E400B3
:1058EE00D600D700FE0807FF507EC000C100D600CC
:1058FE00D700FE0807FF50B2CB00AD00FE0C0BFF29
:10590E0050E4BE00BF00FE0C0BFF511CDA00DB00A2
:10591E00FE0C0BFF50C7CC0000FF50CFCD0000FF98
:10592E00FD104C8C848C848C848C848C8486FE0537
:10593E0000FF107E8C848C848C848C8487FE070000
:10594E00FF10B28C848C848C848C8487FE0700FFBD
:10595E0010E48C848C8487FE0B00FF111C8C848CCD
:10596E008487FE0B00FF10C78C8CFF10CF8C8C8CA5
:10597E00FF504CBC00E4009E00CD00DC00FE060A89
:10598E00FF507ED900C100BA00A000FE0807FF50EC
:10599E00B2C7009D00E500A200FE0807FF50E4BE5E
:1059AE0000BF00FE0C0BFF511CD700D800FE0C0BE5
:1059BE00FF50C7D3D000FF50CFD0D0D1FFFD104C39
:1059CE0000FE23FF107E00FE25FF10B200FE23FF17
:1059DE0010E400FE29FF111C00FE23FF114E00FEF5
:1059EE000FFF504C0CFE23FF507E0CFE25FF50B2D5
:1059FE000CFE23FF50E40CFE29FF511C0CFE23FF6E
:105A0E00514E0CFE0FFF903C00FE0540FE0A00FEBC
:105A1E002840FE0A00FE2A40FE0A00FE2840FE0A2A
:105A2E0000FE2E40FE0A00FE2840FE0A00FE102058
:105A3E00FE28FFFDFDFDFDFDFDFDFDFD104C8A88E0
:105A4E008887FE0C0088888800868CFE0C8600FFF6
:105A5E00107E8A8688888887FE0A00888888008655
:105A6E008CFE0C8600FE03FF10B28A84888887FEA7
:105A7E000B0088888800868CFE0C8600FF10E48A56
:105A8E008884868C87FE0A00FE1AFF111C00FE23F6
:105A9E00FF114E00FE0FFF504C00FE0F0A000000DB
:105AAE00040D00FE0C0C0CFF507E00FE0F0A0000D1
:105ABE0000040D00FE0C0CFE04FF50B200FE0F0D94
:105ACE00000000040D00FE0C0C0CFF50E42457489F
:105ADE005300FE0B0CFE1AFF511C0CFE23FF514E01
:105AEE000CFE0FFF903C00FE0540FE0A0040FE0F2C
:105AFE00004040400040E0FE0C4000FE0540FE0A23
:105B0E000040FE0F004040400040E0FE0C4000FE12
:105B1E000740FE0A0040FE0F004040400040E0FEFD
:105B2E000C4000FE0540FE0A0040FE0F00FE1E4027
:105B3E00FE0A00FE2840FE0A00FE1020FE28FFFD91
:105B4E00104C8A888887FE0C00FF107E8A86888813
:105B5E008887FE0A00FF10B28A84888887FE0B00B1
:105B6E00FF10E48A8884868C87FE0A00FF111C00D1
:105B7E00FE23FF114E00FE0FFF504C31444300FE3A
:105B8E000C0AFF507E265144444D00FE0A0AFF5077
:105B9E00B2214B544400FE0B0DFF50E424574853E2
:105BAE0000FE0B0CFF511C0CFE23FF514E0CFE0F82
:105BBE00FFFD104C8A888687FE0C00FF107E8A86B9
:105BCE00888887FE0B00FF10B28A84888887FE0BB8
:105BDE0000FF10E48A8888888CFE0BFF504C314EF3
:105BEE005300FE0C0CFF507E2651924D00FE0B0B07
:105BFE00FF50B2214B405400FE0B0DFF50E4244DDC
:105C0E00434400FE0BFFFD104C8A8888888887FE6F
:105C1E000A00FF107E8A88868687FE0B00FF10B270
:105C2E008A84888887FE0B00FF10E48A8884868623
:105C3E0088868CFE08FF504C314E54464400FE0AB6
:105C4E0008FF507E3544515300FE0B0DFF50B2211C
:105C5E004B445400FE0B0DFF50E430544853534454
:105C6E005100FE08FFFD104C8A8888888887FE0A3E
:105C7E0000FF107E8A8886888887FE0A00FF10B291
:105C8E008A868887FE0C00FF10E48A8888848688BE
:105C9E008AFE0900FF504C314E52524E00FE0A0849
:105CAE00FF507E354451434400FE0A0AFF50B22194
:105CBE004B5400FE0C0CFF50E43452424851440049
:105CCE00FE09FFFD104C8A88868887FE0B00FF10A8
:105CDE007E8A8886888887FE0A00FF10B28A8888A6
:105CEE008487FE0B00FF10E48A888484868CFE0A6B
:105CFE00FF504C314E494E00FE0B0BFF507E35448B
:105D0E0051434400FE0A0AFF50B22059544B00FE84
:105D1E000B0DFF50E432404B485100FE0AFFFD10C0
:105D2E004C8C848C8487FE0B00FF107E8C848C84BC
:105D3E0087FE0B00FF10B28C848C8487FE0B00FF55
:105D4E0010E48C848C8487FE0B00FF504CC200A1A3
:105D5E0000FE0C0BFF507EC300A100FE0C0BFF508B
:105D6E00B2C400A100FE0C0BFF50E4B200B300FE63
:105D7E000C0BFFFD104C8C848C8487FE0B00FF10E7
:105D8E007E8C848C8487FE0B00FF10B28C848C84F6
:105D9E0087FE0B00FF10E48C848C8487FE0B00FFC3
:105DAE00504CC200A100FE0C0BFF507EC300A100A0
:105DBE00FE0C0BFF50B2DF00A100FE0C0BFF50E4F7
:105DCE00DA00DB00FE0C0BFFFD104C8C8487FE0D01
:105DDE0000FF107E8C8487FE0D00FF10B28C84872E
:105DEE00FE0D00FF10E48C848C8487FE0B00FF50A8
:105DFE004CC200FE0E0DFF507EC300FE0E0DFF5076
:105E0E00B2C400FE0E0DFF50E4D700D800FE0C0BFE
:105E1E00FFFD104C8A8888848488FE0A0088888852
:105E2E000086848688848488888C888C8C8C8600F6
:105E3E00FF107E8A8688888A88848887FE07008875
:105E4E00888800868C8A8C8A8C8A8CFE068600FE58
:105E5E0003FF10B28A88888688888887FE080088A3
:105E6E00888800868C8A8C8A8C8A8CFE068600FF37
:105E7E0010E48A8888888A888487FE080088888843
:105E8E0000868C8A8C8A8CFE088600FE07FF111C09
:105E9E0000FE23FF114E00FE0FFF504C244D464BCB
:105EAE0048524700FE080600000014002853404BDD
:105EBE0048404D4E00FE050CFF507E2551404D755D
:105ECE0040485200FE070900000014007B007C00D1
:105EDE0079007A00FE060CFE03FF50B223445453A1
:105EEE0052424700FE0808000000140099009A0074
:105EFE0079007A00FE060CFF50E424524F40984E73
:105F0E004B00FE080800000014007D007E007F009C
:105F1E00FE080CFE07FF511C0CFE23FF514E0CFE1B
:105F2E000FFF903C00FE0540FE0A0040FE0F0040B1
:105F3E0040400040FE09E0FE044000FE0540FE0A1F
:105F4E000040FE0F00404040004040E040E040E096
:105F5E0040E0FE054000FE0740FE0A0040FE0F0036
:105F6E00404040004040E040E040E040E0FE054060
:105F7E0000FE0540FE0A0040FE0F0040404000407B
:105F8E0040E040E040E0FE074000FE0B40FE0A000D
:105F9E00FE2840FE0A00FE1020FE28FFFDFDFDFD3E
:105FAE00FDFDFDFDFDFD104C8AFE0884FE070088F8
:105FBE00888800868AFE08888C8C8C8600FF107E6E
:105FCE008AFE0884FE070088888800868AFE088C70
:105FDE00FE048600FE03FF10B28AFE0884FE070050
:105FEE0088888800868AFE088CFE048600FF10E4EE
:105FFE0000FE29FF111C00FE23FF114E00FE0FFFB5
:10600E00504C00FE0F0C0000001400FE0E0CFF5052
:10601E007E00FE0F0C0000001400FE0E0CFE03FFAF
:10602E0050B200FE0F0C0000001400FE0E0CFF50CC
:10603E00E40CFE29FF511C0CFE23FF514E0CFE0FEB
:10604E00FF903C00FE0540FE0A0040FE0F0040405F
:10605E00400040FE09E0FE044000FE0540FE0A003E
:10606E0040FE0F004040400040FE08E0FE054000AC
:10607E00FE0740FE0A0040FE0F004040400040FE7A
:10608E0008E0FE054000FE0540FE0A00FE2E40FE22
:10609E000A00FE2840FE0A00FE1020FE28FFFDFD2D
:1060AE00FDFDFDFDFDFDFD504C230D323421FF5055
:1060BE007E233528FFFDA10217FE18FFA30474747A
:1060CE00FFA4047272FFA5047171FFA6047474FF1D
:1060DE00A7047272FFA8047171FFA9047070000505
:1060EE00FE08FFFD810200FE07202322003224332A
:1060FE0033282D2600FE06FF8304393A003124236F
:10610E00002620282DFF8404393A00263124242D20
:10611E00002620282DFF8504393A00212B34240037
:10612E002620282DFF86043B3C00312423002E25FB
:10613E0025322433FF87043B3C00263124242D00D6
:10614E002E2525322433FF88043B3C00212B34249A
:10615E00002E2525322433FF89041A1B00243728EC
:10616E0033FFFDA10217FE18FFA3047070FFA404F5
:10617E007070FFA5047070FFA6047070FFA7047006
:10618E00700005FE08FFFD810200FE073523220088
:10619E0032243333282D2600FE06FF8304393A00BD
:1061AE00222E2D3331203233FF84043B3C0021312B
:1061BE00282627332D243232FF8504101100273470
:1061CE0024FF860410110032203334312033282E60
:1061DE002DFF87041A1B0024372833FFFDC1000052
:1061EE00FE0300FE03A04518000301FFC0031300C9
:1061FE0028FF100080FE0AFF500088FE0AFF900064
:10620E001EFE0AFF101300FF10138CFE1DFF10312F
:10621E008CFE1DFF106D8CFE1DFF108B8CFE1DFF66
:10622E0010A98CFE1DFF10C78CFE1DFF10E58CFE05
:10623E001DFF11038CFE1DFF11218CFE1DFF50133F
:10624E0000FE07254042534E5158002C4E43440049
:10625E00FE0AFF5031002F404D444B0D00FE05321B
:10626E004859440D020800FE023544510D01010249
:10627E0000FF506D002C444C4E51580031444240AA
:10628E004B4B00FE0FFF508B002054534E00224EFE
:10629E004B4E5100FE12FF50A900224E4D5351405D
:1062AE00525300FE14FF50C7002151484647534D2C
:1062BE0044525200FE12FF50E500324F514440430B
:1062CE0000FE16FF510300070601012A003100FEF1
:1062DE00052600FE052100FE0524574853FF5121D7
:1062EE00002457485300FE18FF901310FE1DFF9018
:1062FE003110FE1DFF906D10FE1DFF908B10FE1DC8
:10630E00FF90A910FE1DFF90C710FE1DFF90E51017
:10631E00FE1DFF910310FE1DFF912110FE1DFFFDBE
:10632E00100000FEFB00FEFB00FE57FF500000FEBB
:10633E00FB00FEFB00FE57FF900000FEFB00FEFB85
:10634E0000FE57FFFD10388C8C8CFF503827202D07
:10635E00FF903810FE03FFFD107C8C8CFF507C2EBE
:10636E002AFF907C2020FFFD10978C8CFF50972EDB
:10637E002AFF90972020FFFD2C232C902CFD2D67BB
:10638E002DD62E3A2EA52F102C232C902CFD2D67BA
:10639E002DD62E3A2EA52F102F7F2F7F2F7F2F7FBA
:1063AE002F7F2F7F2F7F2F7F3BB83D263C6D3E9F4B
:1063BE003DE13F543FEB4082429943D9433B453B3D
:1063CE00448745E04673470648BA4978491B4A4315
:1063DE0049DF4AA04B284BB04D904F0B4E4A50A46C
:1063EE004FD6516D523C530B5516564B55B4577EE6
:1063FE0056E6581358A1592F5A425A445A435A46F0
:10640E005A455A475A485A495B4E5C155BC05CD296
:10641E005C745D2D5D825DD75FAC5FAE5FAD5FB0CE
:10642E005FAF5FB15FB25FB360AD60AF60AE60B1E2
:10643E0060B060B260B360B433A9354F347E3708B4
:08644E00362F37DF38BC399905
:10C27600C11402C4000002C2015E01C600011C0115
:03C28600011D6433
:10F08B00E478CBF678C8F678C9F678CAF6C21622B9
:10D7BE00E51D6003151D22051CE51CB41103751C27
:10D7CE0001E51CC454F0440DF524300E3C12E7A0C4
:10D7DE007F0412DBCCE4FB12D81B900E0E12D82560
:10D7EE007B4012D81B900E1312D8257B807D3F7F75
:10D7FE006D12EAA3E51C900E1893FD7F6C12F06675
:0CD80E007B207D5F7F2012EAA3751DFFC8
:10D81A00227D3F7F6D12EAA3E51C2293FD7F6C12E5
:03D82A00F0662283
:10EA7900EF14600714600F2402701E12F08B78C225
:10EA8900760108765E2212F08BD374C878C396E4B7
:0AEA99001896400576000876C822A2
:10D96F0078C3E61846600708E6161870011678C2E5
:10D97F00E6FE08E6FFD374C89FE49E500D78CBE611
:10D98F00604578C276000876C822D374649FE49EFF
:10D99F00501D78C3E664641846702C78CBE670147B
:10D9AF0078A1E6FFF46020EF601D20081A8005784B
:10D9BF00CBE6600878C276000876692278C3E6184D
:08D9CF00467004F6087663229D
:01F1040022E8
:10C8CC0020090302C96712A4DA78A1E6B4FE0812A3
:10C8DC00BE957F0202EA79D3746478C396E4189605
:10C8EC00503A200E057F0112BF8478A1E6FFF46058
:10C8FC0003EF70047B208002E4FB7D5F7F2012EA53
:10C90C00A3E4900F31F012C48630124FE4FD7F3D4A
:10C91C0012F0667B807D7F7F3102EAA378C3E664E8
:10C92C00011846700578A1E6600F78C3E66401181B
:10C93C0046702878A1E6F47022300E1FE4FF12BF77
:10C94C0084C21912EF2512F0157D427F0212F06697
:10C95C0012C96812C9687FFA12F02A227FFA12F003
:07C96C002A7FFA12F02A22D3
:10D39F00900F337401F0900F32F012CBFC12E99C16
:10D3AF0012F1047FFA12F02A7FFA12F02A7E327FEE
:10D3BF00CE12D50E12E81012F10312B39640F530CB
:10D3CF0010F212A67A78A5EFF612CEEE40E612E82A
:10D3DF00AE40E112EA4E78A1E6FFF46003EF700D64
:10D3EF0030090AE56F30E50512D7BE801378A1E644
:10D3FF00600BE56F30E506536FDF02ED8712D96FD3
:0BD40F0078A5E6FF12C8CCC21080A96F
:0EC2890001CF00C11501CC0001CD0001CE0097
:10EF7300AF647D331286D678C4A60608A607227826
:09EF8300C8F678C9F678CAF62236
:10EA2200E4FF20B4027F0820B503430760900F384B
:10EA3200E020E003430720900F34E020E003430787
:0BEA420010900F35E020E003430701B7
:01EA4D0022A6
:10A67A00E4F52478CDE618F612EA2208A607300F88
:10A68A0025E630E460186630E45B12A7E418663009
:10A69A00E411E56F20E30330E506536FF712ED8707
:10A6AA007F81227F002278CDE6B41805436F0880A7
:10A6BA000E78A1E6700F78CDE6B47009436F2012C8
:10A6CA00ED877F802278CDE630E41A186630E412EE
:10A6DA00E478CFF612A7E4186630E4037F80227F7D
:10A6EA0000227F002278CDE6FF14603024F96077DB
:10A6FA0024E8603E24C0606F244C600302A7DA7825
:10A70A00CCE66F5414700302A7E112EA2278CDEF67
:10A71A00F670F778CFF675240902A7E179CCE778C5
:10A72A00CD6620E00302A7E1E478CFF6752405029E
:10A73A00A7E179CCE778CD6630E513E478CFF6FE69
:10A74A00FC12EF7375240278CE767802A7E178CEF0
:10A75A00E660041602A7E178CBE6607BE478C4F6EB
:10A76A0008F6752482807078CBE660097E007C004A
:10A77A0012EF73801030160DE56475F004A479C5E4
:10A78A00F7E5F019F778CDE6FF18665F6018E47808
:10A79A00CFF678CDE6B408047F0380027F048F24C5
:10A7AA0078CE760F803178CEE66003168029740F52
:10A7BA00D378CF964006061876018004E478CEF660
:10A7CA0078CDE6B408047F0380027F048F248007D3
:09A7DA0078CE760FE408F6AF24F6
:0EA7E300227F1412F02A12EA2278CDEFF6221D
:10A4DA008F2430143DC21412A64312C97378CBE6F6
:10A4EA006005752483802BE4F524FB12A6587B4073
:10A4FA0012A6587B807D3F7F6D12EAA3E4FBFD7FA5
:10A50A006C12EAA3C374C878C396E418965003126F
:10A51A00DFA878CBE6702220161F78C3E664C81835
:10A52A0046700812A64312C973802078C3E6646491
:10A53A001846701712D5F78012E524700E78C5E612
:10A54A0018467007E5646003752482E524146029BF
:10A55A0024E760252498706078CBE67006201603FD
:10A56A0002A642E478CBF612EF82C21612A6721243
:10A57A00A6687E327FE502C973E55F540770047FDF
:10A58A00018032E55F5407FFBF01047F028026E5A0
:10A59A005F5407FFBF02047F03801AE55F5407FF79
:10A5AA00BF03047F05800EE55F5407FFBF04047FE5
:08A5BA00058002E4FF02ECDD64
:10A5C20078CBE6F525AF2412BB7878CBE6FF65257C
:10A5D2006037EF6026E525701612A6727B017DFFBB
:10A5E2007F2012EAA312A6687E327FE512C9737F2A
:10A5F2008312BB78E525704802D9D7E412EF827D39
:10A60200407F0212F06602E31A78CBE6602EE52460
:10A61200B483107E327FCE12D50E7B017DFE7F6D1C
:10A6220012EAA3E52464036005E524B40412E4FD00
:10A632007F0112F066E4FD7F1F02F066E478C0F647
:10A64200227D407F0212F066E4FB7DFE7F6D12EAFE
:10A65200A37E327FE5227D3F7F6D12EAA3E4FBFDFC
:10A662007F6C12EAA322E4FB7DFE7F6D12EAA32235
:08A672007D407F0212F0662218
:10C2970001CB0001C80001C90001CA0001C700C1E4
:01C2A7001680
:106A670078C9E614F91313543F75F0AAA4FFAEF0E2
:106A77002496FDE43EFCEF241AFBEE3401FAE954B8
:106A87000375F021A4FFAEF02436F582E43EF583CA
:106A9700EF2454F534E43EF533858331858232752E
:106AA700350175360175370E7538FBE4F539753ADA
:106AB70001753B192278C8E6FF7E007C007D211214
:106AC70086D6EF2415FDE43EFCEF2433F534E43E8F
:106AD700F5338C318D32E4F535F53675370E75386B
:106AE700FBF539753A01F53B7D967B1A7A01FC7FF8
:106AF70006227890E6FB7A00C3E5539BFFE49AFEF3
:106B07007C007D321286D6C374809BFDE49AFC120A
:106B170086E88F2F75306475310275320E7B117DD3
:106B27001F22EF25E0FDEE33FCC374E89DFB7401E3
:106B37009CFA18E6FE08E6FF8E31F532C374089F0B
:106B4700F53474019EF533E4F535F53675370E7572
:106B570038FBF539753A0122856B2F7530FF753192
:106B67000275320E7B117D242278C9760274027574
:106B7700F007A4241DFD7538207539022278C8E670
:106B8700FF7E007C007D211286D6EF2415FDE43EB2
:106B9700FCEF2433F534E43EF5338C318D32227823
:106BA700C87601E408F6F531753236F53375345495
:106BB70075350175360175370E7538FB2278C9E6CC
:106BC70075F007A4241DFD753840753902227890A9
:106BD700E6FB7A00C3E5539BFFE49AFE7C007D3217
:106BE7001286D6C374809BFDE49AFC1286E88F2F29
:106BF70075306475310422750C05E4F50D750E903A
:106C07002278C9E614F91313543F75F0AAA4FFAE0E
:106C1700F02496FDE43EFCEF241AFBEE3401FAE97A
:106C2700540375F021A4FFAEF02436F582E43EF557
:106C370083EF2454F534E43EF5338583318582327E
:106C47002225E025E004FEC454F04FF50F08E62D99
:106C5700F510E4F5117F0C22788DE6FFC39552F508
:106C67002FC3EF788C96F53022750C06750D0175DC
:106C77000E9222C3E562950CF52FC3E50D950CF531
:106C87003022C3E563950EF52FC3E50F950EF5305A
:106C970022E92401FFE433FEE6FCC39FEE6480F89B
:106CA70074809822E555547C1313543FF52F7530A3
:106CB7001F22856B2F7530FF75310422E530A4FD47
:106CC700ACF0E534C4F8540FC868FFE533C454F09A
:106CD70048FE1286E88F31E4F533F53422F583E474
:106CE70093FE740193FF22740FD378CF96227531E8
:106CF7000075323675330075345422902B6793260E
:106D0700F618E436F622E55E540775F002A42278F9
:106D1700C9E675F003A4242122A907760008761393
:106D270008760122E4FB7DFE7F6D22C3741F956CFC
:106D3700F52F75301F22752E13752F0222752E1011
:106D4700752F0222E993FFFBED2401F582E433F569
:106D570083D3E5829B7480F86583982226E41836EE
:106D6700540F4450F50F08E6227B88FA7D0AFC7F12
:106D77000522E55F54E0C4135407F52F7530072249
:106D8700752C13AB567D0C7F0522752C13AB577DE5
:106D97000C7F0622752E23752F02227B017DFE7F35
:106DA7006D22E478C8F608F6227583002BFBE5838D
:106DB7003AFAD3EB9F7480F86A982275F003A4C55A
:106DC7008325F0C58322E625E0FD18E633FCC3746E
:106DD700E89DFB74019CFA2275F00AA4FFC3227593
:106DE70032027B117D1F7F052275320C7B117D1FBF
:106DF7007F07227532037B117D1F7F0922752C13B4
:106E0700AB707D0C7F0722ED26E41836540F22E580
:106E170030A4FFAEF0C3E5349FE5339E22D3EF9550
:106E270062EE956122750FC1E52C25E025E02275FC
:106E3700388CE4F5392278C9E675F005A4241F22B9
:106E4700E55424B2F52F227B00AD2B02D754FFE582
:106E57000E34FEFEEF7802222401FFE433FE22E423
:106E6700F538753901227C007D641286E88F31225E
:106E77007B007A00795702D7547B0E7D247F092245
:106E870085582F7530647531022285592F75306406
:106E970075310C22855A2F7530647531032275F0D0
:056EA70008A4241C22D8
:10DD4100AE07E55F540714601A14602414602E14A2
:10DD51006038240470417405D39E50037F0122EE84
:10DD610004FF227405D39E50037F0122EE04FF229B
:10DD71007405D39E50037F0122EE04FF227405D364
:10DD81009E50037F0122EE04FF227405D39E5003AF
:0ADD91007F0122EE04FF227F012231
:10DD9B00AE07E55F540714601A14602414602E1448
:10DDAB006038240470417401C39E40037F0522EE4A
:10DDBB0014FF227401C39E40037F0522EE14FF2241
:10DDCB007401C39E40037F0522EE14FF227401C32E
:10DDDB009E40037F0522EE14FF227401C39E400375
:0ADDEB007F0522EE14FF227F0122C3
:10B4BF008F2C8C2D8D2E8A2F8B30E52CD39407401B
:10B4CF000302B5E6126BFE126E2C126C5712E4D902
:10B4DF00126C70E535540733333354F8FFE53654A7
:10B4EF00074FF50F853810853911E4F5127F0C12CF
:10B4FF00E4D9126BFE750FE1126E2F04126C571206
:10B50F00E4D9750C09126C737E00E52E543F780256
:10B51F00C333CE33CED8F9F50FE52D5407FEE52E04
:10B52F0054C07806CEC313CE13D8F9FD7E00E53292
:10B53F0054077805C333CE33CED8F94DF510E53126
:10B54F005407FEE53254F87803CEC313CE13D8F95F
:10B55F00F5117E00E530543F7802C333CE33CED899
:10B56F00F9F512E52F5407FEE53054C07806CEC327
:10B57F0013CE13D8F9FD7E00E53454077805C33395
:10B58F00CE33CED8F94DF513E5335407FEE53454D9
:10B59F00F87803CEC313CE13D8F9F514E4F5157F5D
:10B5AF000C12E4D97F1912F02A126BFE126E2C24A2
:10B5BF0003126C5712E4D9126C70E4F50FE53A548C
:10B5CF0007C454F0FFE537540F4FF510853B11E4D6
:08B5DF00F5127F0C12E4D922E1
:02D66B008B2D05
:10D66D0078A6126D2078A8126C98500FEC902B7A3A
:10D67D009378A7126D0678A80680EA126BFE902BA0
:10D68D007B126D4B5049ED2401FBE433FAE52D126D
:10D69D006DB04008E9902B7B939DF52D78A7126E08
:10D6AD000EFFE52F126C4812E4D9E52FB40308E5FF
:10D6BD002D75F003A48002E52D2403FF8F0C750D4D
:0FD6CD0002750E92852E0FE4F5107F0C12E4D932
:01D6DC00222B
:10EB42008F278D288B29852A2AE5286019E52790A9
:10EB52002B7B93FBE4F52E752F03AD29AF2712D63D
:07EB62006B0527D528E7220F
:02C607008D2A7A
:10C6090078A6126D22EF2401FDE433FC78A8E6F93F
:10C61900C39DEC126CA4500FE9902B7A9378A71262
:10C629006D0678A80680DEEB75F06484F51675F062
:10C6390064A4FFC3EB9F75F00A84F517E51675F03E
:10C6490064A4FFC3EB9FFFE51775F00AA4FEC3EFCF
:10C659009EF518E5166006051605178006E51760AC
:10C669000205170518126BFEE52A78A7126D6325D6
:10C679002A126C5712E4D9126C7085160F8517109F
:10C68900851811E4F5127F0C12E4D9126BFEE52A24
:10C6990078A7126E0F4490F50F08E6252A126C57F9
:10C6A90012E4D9126C70852C0F852C10852C11E49D
:07C6B900F5127F0C02E4D929
:10D89B00ED6404702C30151712867EFFE52D14FEF7
:10D8AB00EFC39E5006EF2402FF804AAF2D80461235
:10D8BB00867EFFC3952D5005EF04FF8002AF2D80B0
:10D8CB003430152112867EFFE52E2401FDE433FC56
:10D8DB00D3EF9DEC126CA4400812867E24FEFF80D1
:10D8EB0002AF2E801012867EFFD3952E4005EF14CB
:0AD8FB00FF8002AF2EEF1286C42258
:10DB0900ED6404703012867EFF740FD39F4053205A
:10DB1900150F740FD39F4005EF04FF80417F0F80DD
:10DB29003D12867EFF740ED39F4006EF2402FF80CC
:10DB3900027F0F802912867EFF602720150EE4C31D
:10DB49009F5005EF14FF80027F00801212867EFF2E
:10DB59007401C39F5006EF24FEFF80027F00EF127D
:03DB690086C4224D
:10E522007F2912E559E4250F126E55CEC313CE137F
:10E53200D8F904F5317530097F3412E559E50F2415
:10E54200EC126E55CEC313CE13D8F985300C85313B
:06E552000D750E03F50F2C
:10E5580022E4FB7D0212ED44E50D5407F50E850C0F
:02E568000F2280
:10CE61008F2F12E522D3E50C9562E495615018C32A
:10CE7100E50D9562E49561400EE50ED3956350078B
:10CE8100E50FC39563500C7563607561007562654C
:10CE910012E96E78CBE6B40F097561007562E6752B
:10CEA10063647F2012DBCC126BFE750FC0F5107529
:10CEB1001106751201751392E563C313F514E5624A
:10CEC100AE617802CEC313CE13D8F9F515E56254DD
:10CED10003C4333354C0FFE5635401FEC43354E04B
:0DCEE1004F452FF516E4F5177F0C02E4D93C
:02D82D008B3737
:10D82F0078A9126D2078AB126C98500BEC78AA1275
:10D83F006D0278AB0680EE126BFE902B68126D4B6B
:10D84F005049ED2401FBE433FAE537126DB040087F
:10D85F00E9902B68939DF53778AA126E0EFFE53984
:10D86F00126C4812E4D9E539B40308E53775F003B3
:10D87F00A48002E5372403FF8F0C750D02750E92FD
:0BD88F0085380FE4F5107F0C12E4D97F
:01D89A00226B
:069212008F2C8D2D8B2E28
:1092180078A6126D22E52C126E5F78A8E6FD126C16
:10922800A1500BED78A7126D0278A80680E774FBB1
:10923800252EF52EFF7E007C007D061286D6EF24B3
:10924800FAFFEE34FFFEAD2F1286D68E338F3475BB
:109258000C06126C01E52D78A7126E0F4490F50FDD
:1092680008E6252DF510E531C454F0F511E4F512A2
:109278007F0C12E4D9750C05126C73E531C454F0F7
:10928800F50F126C5712E4D9E52D2405FDE532C41B
:1092980054F0F5387539027B0CAF2C12D82D750CAB
:1092A80006126C01F512F52CE52CC3952E4003022D
:1092B80093E8E52D78A726FFE41836FE7C00EF2515
:1092C8002CFFEC3ECF2405CF3400126D67252D25E9
:1092D8002C2405F510E52C600AE52E14652C600396
:1092E80002936FE5344533606F75F003126E1640D4
:1092F80010E52C70047D1380027D1E8D11C302932E
:109308008075F003126CC37404D39531400FE52CBB
:1093180070047F1080027F1B8F110293DE7408D3C4
:109328009531400FE52C70047F1180027F1C8F114E
:109338000293DE740CD39531400FE52C70047F1234
:1093480080027F1D8F110293DEE52C70047F13804D
:10935800027F1E8F110293DEE52C70047F108002BD
:109368007F1B8F110293DEE5344533606675F00686
:10937800126E16400F75111AE5349FF534E5339EC9
:10938800F533805275F006126CC304D39531400250
:1093980080417404D39531400575111580387406E1
:1093A800D395314005751116802C7409D395314039
:1093B800057511178020740BD39531400575111868
:1093C8008014740ED39531400575111980087511F4
:1093D8001A80037511147F0C12E4D9052C0292B07F
:1093E800E52F75F00A84F530126DDFE52F9FF52C17
:1093F800E53075F00A84F531126DDFE5309FF53000
:10940800052C7004E5316006E53004FF80027F001A
:109418008F30E531600404FF80027F008F31126BCA
:10942800FEE52D78A7126D63252D126C5712E4D92D
:10943800126C7085310F853010852C11E4F5127F80
:049448000C02E4D955
:10EDE7007F0112CE617532017B0F7D0B7F0512EB20
:0FEDF7006978CBE6B401077E327FEC12C9732234
:10E3B1008B2B8A2C892D12EDE77E337F3812C9739E
:10E3C100126D0D2446F582E5F03464126CE412C935
:10E3D10073AE2CAF2D12C97375F010E52EA424B6BF
:10E3E100F582E5F03463F583E55E540775F00212BA
:0BE3F10088CF126CE612C973029FDD9A
:10EB69008F2F8D308B31853232E5306019E52F904A
:10EB79002B6893FBE4F538753903AD31AF2F12D803
:07EB89002D052FD530E72216
:06D74E007B007A00795611
:10D75400ED6404703412867EFF7464D39F405A12C1
:10D764006CEE40117464D39F400712867E04FF80E0
:10D77400447F64804012867EFF7463D39F4006EF2B
:10D784002402FF80027F64802C12867EFF602A12AE
:10D794006CEE400FE49F500712867E14FF80027FD8
:10D7A40000801212867EFF7401C39F5006EF24FE90
:0AD7B400FF80027F00EF1286C422FE
:10E0A2008F2978C8E6FF6034E529B4030FEDB50780
:10E0B200047F01801778C8E604FF801078C8E6FF65
:10E0C200B40106AE05AF068003EF14FF78C8A607B9
:10E0D200126B84126AA6126AEF02B4BFE52978CBEA
:10E0E200B40308E6FF12DD41A60722E6FF12DD9B1C
:03E0F200A607225C
:109FDD00126E667B0F7D0C7F0312D82D78A6126D45
:109FED002278A8E6FFC39404500EEF902B679318C8
:109FFD00126D0678A80680E9126BFE78A7E6240C90
:10A00D0018E4126D66240C126C5712E4D978A1E68F
:01A01D00FF43
:10A01E007881E6F52F08E6F530E55F54077065EFB9
:10A02E00B42E02801E78A1E6FF742ED39F401074CA
:10A03E0027D39F5002801A7423D39F50288020EF7D
:10A04E00B43B08752F06753040801A7439D39F5073
:10A05E0008752F05753000800C7437D39F50067528
:10A06E002F0475308078A1E6FF64086004EFB40910
:10A07E0013E55E30E408752F027530808006752F6B
:10A08E00027530D0750C0C126C73AE2FAF30126E91
:10A09E006D740AD39531500B750F02E53124F7F527
:10A0AE00108008E4F50FE53104F510E53175F06424
:10A0BE00A4FEC3E5309EF53175F00A84F511126DDC
:10A0CE00DFE5319F04F512051175130E7886E6FE55
:10A0DE0008E6FF126E6D7887E6FFE53175F064A431
:10A0EE00FEC3EF9EF518740AD395315026750C0DEC
:10A0FE00751402E53124F7F515E51875F00A84F5A7
:10A10E0016126DDFE5189F04F5170516E4F518F520
:10A11E0019801DE53104F514E51875F00A84F5155E
:10A12E00126DDFE5189F04F5160515E4F517F51801
:10A13E00E4F5187F0C12E4D9750C07126C7378973E
:10A14E00E6FF75F00A84F50F75F00AA4FEC3EF9EC4
:10A15E0004F510050F751127751259E4F5137F0CD0
:10A16E0012E4D9740AD395315009126E367B017DF3
:0FA17E00158007126E367B017D147F0312D82DDA
:01A18D0022AF
:09F0C20078CB760F78C8760122A4
:10D905008F282016257F0112CE617E307FA412C993
:10D9150073126D0D2484F582E5F03431126CE41236
:10D92500C973126DA212EAA3D216E5286404700B1E
:10D93500E56CD394004013156C800FE528640370E3
:10D9450028E56CC3941F5002056C12EEB612ED87E4
:10D95500C3741F956CF52C752D1F752E04752F0E30
:0AD965007B187D07E4FF12944C22AA
:10EE4300E56F78CB30E30C760F78C87601E408F6EB
:0DEE530008F6227601126DA908F6C21622FB
:10F05300E55F5407700C78CB760878C8760108F61C
:03F0630008F6228A
:10B13D0078C8E6701A78A1E6700302B269F470035C
:10B14D0002B269126BA6126AB3126AEF02B4BF782B
:10B15D00C9E6FF606618E614602614603014604975
:10B16D0024FC60392402704EEFB4010B12E0F5BFE0
:10B17D00FC0578A176FE22126BC47B047F0D803313
:10B18D0085562F126BF7126B217F05800B85572F7C
:10B19D00126BF7126B217F071292128019126E3DFE
:10B1AD00126BCD7B047F0B800A126D16126BCD7B5B
:10B1BD00017F0912D82DE478C9F62278C8E6FF641C
:10B1CD0006700CFEFC126AC412B4BF126DA922786F
:10B1DD00A1E6700302B269F4700302B26978C8E6A1
:10B1ED0014601A14602514604A14605E24FD602AF0
:10B1FD0024027068126B707B047F0D804A78C976CB
:10B20D000185562F126B1B7F05800C78C976018541
:10B21D00572F126B1B7F07029212E55F5418131301
:10B22D0013541F0478C9F6126E40126B7C7B047F99
:10B23D000B8014E55EC41354030478C9F6126D191E
:10B24D00126B7C7B017F0902D82D126ABC12B4BF30
:0DB25D0078C97601E408F67F8312EBDC224D
:10B26A008F2878C9E6700302B38E18E614603C147E
:10B27A00605914700302B34524FC6065240260031C
:10B28A0002B395E528B403047F0180027F0278C9DE
:10B29A00A607126BCE7B0E7D247F0D12D82D78C99E
:10B2AA00E6126B767B047F0D02D82DAD2812D74E9D
:10B2BA0085562F126B1B7F05129212E55F54077099
:10B2CA000512C2F6801812BA678013AD28126E777B
:10B2DA0085572F126B1B7F0712921212BA6702E967
:10B2EA00F6E528B4041278C9E6FFB404067E047FA2
:10B2FA00048015EF04FF801078C9E6FFB401067ECA
:10B30A00017F018003EF14FF78C9A60778C9E61404
:10B31A0033333354F8FFE55F54E74FF55F126BCED2
:10B32A007B147D247F0B12D82D126E3D126B7C7B11
:10B33A00047F0B12D82D12BA678046E528B4040D93
:10B34A007404D378C996404378C906800B7401C344
:10B35A0078C996503678C91678C9E614C43354E0C9
:10B36A00FFE55E549F4FF55E126BCE126E8012D8C7
:10B37A002D126D16126B7C7B017F0912D82D12E5F6
:0CB38A006A02E96E7D06AF2812E0A222E4
:10E3FC007BFF7A3A796AE4F52EFF12E3B1126CF5E1
:10E40C00126AA6126D7012B4BF85562F126BF712DA
:10E41C006B217F0512921285572F126BF7126B210D
:10E42C007F0712921278C8E6FF24FC700C126B88DE
:0AE43C00126AA6126AEF12B4BF22A2
:10D2A60078CB760778C9E66404701018126ABE1245
:10D2B600B4BFE478C9F608F602D31F78CAE6602739
:10D2C600E4F618E624FE600F1460142402704A8502
:10D2D600582F126BF7802C85592F126BF7802C85EF
:10D2E6005A2F126BF7802C78A1E6602DF4602A780D
:10D2F600CA760118E624FE600F1460142402701921
:10D30600126E87126DE6800E126E91126DF0800617
:0ED31600126E9B126DFA12921278CB760122E3
:10D006008F2B78CB760718E6604718E624FE601665
:10D01600146022240270327A007958126E4E126E13
:10D0260087126DE680207A007959126E4E126E9143
:10D03600126DF080117B007A00795AAD2B12D7540D
:10D04600126E9B126DFA12921212BA6712E9F680EC
:10D0560035E52BB4031078C9E6FFB404047F0180DC
:10D0660013EF04FF800E78C9E6FFB401047F048045
:10D0760003EF14FF78C9A60778C9126B86126AA651
:0BD08600126AEF12B4BF78CB760122D3
:10DEA7007BFF7A5A794A752E06E4FF12E3B1126CAA
:10DEB700F5126AA6126AEF12B4BF78A1E66003B43E
:10DEC700FF04E478CAF678CAE6702B087607855807
:10DED7002F126BF7126DE612921285592F126BF7FC
:10DEE700126DF0129212855A2F126BF7126DFA12F9
:07DEF700921278CB760122A4
:10BD910078C8E6701A78A1E6700302BE94F47003C5
:10BDA10002BE94126BA6126AB3126AEF02B4BF7894
:10BDB100C9E6605918E624FE601A14603E14601E3C
:10BDC10014602824047041126C5F753104126B21D8
:10BDD1007F058022126BD5126B217F078018126CB0
:10BDE100AB753104126B217F0B800B126E47126B06
:10BDF100F7126B217F0D129212800D126D16126BCC
:10BE0100CD7B017F0912D82DE478C9F62278C8E6E6
:10BE1100FF6406700CFEFC126AC412B4BF126DA955
:10BE21002278A1E6606DF4606AE55F5407600778E7
:10BE3100C8E66403705D78C8E624FE601B146040A8
:10BE410014602014602B2404704978C97601126CA7
:10BE51005F126B1E7F05802578C97601126AF97F12
:10BE610007801A78C97601126CAB126B1E7F0B80AA
:10BE71000C78C97601126E47126B1B7F0D0292126C
:10BE8100E5600478C9F6126D19126B7C7B017F099C
:04BE910012D82D2274
:108FD0008F2878C9E6700302920A18E624FE70030F
:108FE00002909314700302919B1470030290D014AA
:108FF000700302910624046003029211E5286404C0
:109000007045788CE6FFC395524003029211126CB2
:10901000EE4014E552D39F4006E55214FF800478D9
:109020008CE6FF8F52805B788CE6FF2402FDE433F0
:10903000FCE552D39DEC126CA44008E55224FDFEE1
:10904000FF80008F52803B788DE6FFD3955250030E
:10905000029211126CEE4013E5529F5006E5520445
:10906000FF8004788DE6FF8F528017788DE6FF240D
:10907000FEFEE552C39E5008E5522403FEFF800029
:109080008F52126C5F126B1E7F0512921212DB6CF4
:109090000290FEE528B4041D7890E6FFC3E49FFF2C
:1090A00074019400FED3EF9553EE940050030292A6
:1090B000110553800D7890E6C39553400302921139
:1090C0001553126AF97F0712921212C77702919410
:1090D00053557CE528B4040E747CD3955550030297
:1090E000921174048009E555700302921174FC25F5
:1090F00055F555126CAB126B1E7F0B129212AF55C9
:1091000012B94A029194E5286404704374B2D3956D
:10911000545003029211126CEE401574B1955440F4
:1091200007E554126E5F80047E007FB28F54801773
:1091300074B0C39554400AE5542402FFE433FE8022
:10914000047E007FB28F5412989912DB6C803A74BF
:109150004EC395544003029211126CEE4013744FAB
:10916000D395545006E55414FF80027F4E8F5480EF
:10917000127450D395545007E55424FEFF80027FAB
:109180004E8F5412DB6C129899126E47126B1B7F34
:109190000D12921278A1E6FF02E848E528B4040D0A
:1091A0007405D378C996406978C906800B7401C3E9
:1091B00078C996505C78C916126BCE126E8012D8A0
:1091C0002D126D16126B7C7B017F0912D82D78C988
:1091D000E614F56012DCE77882E6B4001018E6B415
:1091E000050BE560B402067B017DFF80157882E601
:1091F000B4001418E6B4050FE56064026009E4FBEE
:109200007DFE7F1512EAA302E96E7D06AF2812E00B
:02921000A22298
:10D495007BFF7A41793E752E017F0112E3B175312B
:10D4A50000753257753300753475126AA6126D70A2
:10D4B50012B4BF78A1E66003B4FF03126DA9E55F5E
:10D4C5005407600A78C8E664036003E408F678C97F
:10D4D500E67035126C5F753104126B217F0512926F
:10D4E50012126BD5126B217F07129212126CAB755B
:10D4F5003104126B217F0B129212126E47126BF7D9
:09D50500126B217F0D029212222B
:10817E0078C8E670087601126BAB0282B778C8E653
:10818E0024FE602614604A14606E14700302834E3F
:10819E0014700302836F24056003028378E55E5436
:1081AE00070478C9F67F8302EBDC78C9E6600DE43C
:1081BE00F612E522126C7A753104800D78C97601BB
:1081CE0012E522126C7A753102126B217F0702833F
:1081DE006C78C9E6600DE4F612E522126C897531F1
:1081EE0004800D78C9760112E522126C8975310270
:1081FE00126B217F0902836C78CAE670030282C07B
:10820E00E4F618F6126BCE1283F5126E661283F533
:10821E0075388A1283CC126E661283E3E55E5407BC
:10822E0024FA60151460202402703C128395753870
:10823E00B31283797538C980251283957538DB1290
:10824E0083797538E58017126E367D251283ED75AC
:10825E00389B1283A5126E361283D975389C7539E8
:10826E00017B017D2B802475382E1283A575382D48
:10827E007539017D261283ED75382E7539011283FD
:10828E00D97538257539017B027D2C7F0B12D82DBF
:10829E00126BCE1283E3E4F5381283B2E4F5381292
:1082AE0083BF126B84126BB7E4126AB3126AEF02C9
:1082BE00B4BF78C9E6FF6070B4020F126BC67B03C1
:1082CE007F0B12D82DE478C9F62278CA7601E564C0
:1082DE00C39405500D75641478C476030876FC12A9
:1082EE00E96E7538E07539027B0C7D247F0B12D850
:1082FE002D75388C1283CC126BCE7B017D237F0BB8
:10830E0012D82D75380D1283B2126BCE7B017D30D3
:10831E007F0B12D82D75380C1283BF85642F7530E4
:10832E003C126B1E7F0B8036E56460047F01800279
:10833E007F0278C9EFF6126B767B037F0B02D82D86
:10834E0078C9E6600AE4F6126D79753104800A7810
:10835E00C97601126D79753102126B217F0D029271
:10836E0012126ABC12B4BF126DA9227539017B01BB
:10837E007D257F0B12D82D75388CE4F5397B017D68
:10838E002B7F0B12D82D2275388CE4F5397B017DAD
:10839E00257F0B12D82D227539017B017D257F0B90
:1083AE0012D82D227539017B017D237F0B12D82D1A
:1083BE00227539017B017D307F0B12D82D22E4F519
:1083CE00397B0C7D247F0B12D82D227B017D2B7FD8
:1083DE000B12D82D227B0C7D247F0B12D82D227BE5
:1083EE00017F0B12D82D227B037D1F7F0B12D82D00
:0183FE00225C
:108D81008F2878C9E67003028FC818E624FD7003A6
:108D9100028E57147003028EE6147003028F64244E
:108DA100036003028FCF12E522E5286404704CAF03
:108DB1000DFE126E245003028FCF126CEE4017127B
:108DC1006E24400CE5622401FFE43561FE028E4809
:108DD100AF0D7E008071AF0D7E00EF24FFFDEE34FC
:108DE100FFFCD3ED9562EC9561400EE5622402FD36
:108DF100E43561FCFEAF058000804CAF0C7E00C302
:108E0100126E254003028FCF126CEE4017126E25B1
:108E1100500CE56224FFFFE56134FFFE8004AF0CD6
:108E21007E008023AF0C7E00EF2401FDEE33FCC3F6
:108E3100ED9562EC9561500FE56224FEFDE561342C
:108E4100FFFCFEAF0580008E618F62126C7A126B9F
:108E51001E7F07028EDB12E522E52864047037E5E8
:108E61000FD395635003028FCF126CEE4013E50FC1
:108E7100D395634006E56304FF8002AF0F8F6380E3
:108E810051E50F14D395634007E5632402FF800287
:108E9100AF0F8F63803CE50EC395634003028FCF14
:108EA100126CEE4012E50E95635006E56314FF80E7
:108EB10002AF0E8F63801BE50E126E5FC3EF9563E9
:108EC1007480F86E985007E56324FEFF8002AF0EB0
:108ED1008F63126C89126B1E7F091292127F01122D
:108EE100CE61028FC5E5286404702078CAE6600F60
:108EF100E564B43C047F3C8024E56404FF801E7873
:108F0100C9E6604B7602E4F564802B78CAE6601FFF
:108F1100E564B405047F058004E56414FF8F64856E
:108F2100642F75303C126B1E7F0B129212802078D9
:108F3100C9E6601B7601126BCE7B0E7D247F0B127E
:108F4100D82D78C9E6126B767B037F0B12D82DAF33
:108F5100647E007C007D331286D678C4A60608A6FE
:108F6100078061E55F54E0C4135407F50CE52864FC
:108F710004701478C9E6602FE50CB407047F0780FC
:108F810016E50C04FF801078C9E6601BE50C700340
:108F9100FF8004E50C14FF8F0CE50CC43354E0FF93
:108FA100E55F541F4FF55FE50C33333354F8FB7D18
:108FB100C77F6D12EAA3850C2F753007126B1E7FD8
:0F8FC1000D12921202E96E7D06AF2812E0A22275
:10D6DD007BFF7A4C793F752E037F0212E3B17531D2
:10D6ED0000753278753300753496126AA6126D7016
:10D6FD0012B4BF78C9E6704812E522126C7A753102
:10D70D0004126B217F0712921212E522126C897599
:10D71D003104126B217F09129212126D7975310449
:10D72D00126B217F0D12921278C8E6B4010C126CA7
:10D73D00F5126AA6126AEF12B4BF126DA202EAA325
:01D74D0022B9
:10DE4E00E55E5407FF78C9E614FE6F6047EE54078F
:10DE5E00FFE55E54F84FF55E12E96EE55E54072459
:10DE6E00FA60071460162402702A126D2B12EAA3B0
:10DE7E007E147F087B457A007DA98010126D2B12CF
:10DE8E00EAA37E0E7F1D7B4B7A007D737C0512C04C
:09DE9E007012D6DDE478C9F62209
:10E6B2008F2B126C08126B4EF53B7F0612B4BFE52E
:10E6C2002BB4031078C9E6FFB408047F018013EF6E
:10E6D20004FF800E78C9E6FFB401047F088003EFCF
:0EE6E20014FF78C9A607126A677F0602B4BF4C
:10EE60007BFF7A5E7920752E077F0312E3B17E5F08
:0DEE70007FAB12C973126A677F0602B4BF40
:109C700078C8E67026760108F6F531753236F53388
:109C8000753454753501753601126AE212B4BF128B
:109C90006CF5126AA6126AEF02B4BF78C8E624FE19
:109CA0006055147003029D81147003029DFC1470B2
:109CB00003029E2024046003029E29E55F5407F5F9
:109CC0000CB401047F028026E50CB402047F0380FB
:109CD0001DE50CB403047F048014E50CB404047F78
:109CE00005800BE50CB405047F0680027F0178C96E
:109CF000A6077F8302EBDC78C9E66069126EA512C5
:109D00006BCD7B077F0712D82D78C9E6B401047F9D
:109D10000080027F108F0CE55E54EF450CF55EE489
:109D200078C9F612E96EE55F54076003029E297850
:109D300087E66490700418E664016003029E297847
:109D4000A1E6FF64057003029E29EF6433700302ED
:109D50009E29E55E30E406535EEF76FE22435E10F8
:109D600078A176FE22E55E30E4047F0280027F0166
:109D700078C9EFF6126EA5126B7C7B077F07029DF8
:0B9D8000F978C9E6FF606B64017058C1
:109D8B00E55E5407F527E55F5407F5287407C3957F
:109D9B00275003E4F52778C4760408760012CDCA61
:109DAB00E564F8E479C5F7E825E019F7E55E54F8C2
:109DBB004527F55EE55F54F84528F55F12E96E120D
:0A9DCB00BA6712EEB67F0112CE61F6
:109DD50012CA1878A1E6FF12EB1B78A176FE126B6A
:109DE500C47B047F0912D82DE478C9F622126B7062
:109DF5007B047F0902D82D78C9E6600AE4F6126D66
:109E050032753104800D78C97601536C1F126D329D
:109E1500753102126B217F0B029212126ABC12B4C9
:059E2500BF126DA9222F
:10CD32008F2878C9E6700302CDC218E624FD60345C
:10CD42001460562402600302CDC9E528B404047FAE
:10CD52000280027F0178C9A607126BCE7B107D2468
:10CD62007F0712D82D78C9E6126EA5126B7C7B075D
:10CD72007F078022E528B403047F0180027F0278C6
:10CD8200C9A607126BCE126E8012D82D78C9E61290
:10CD92006B767B047F0902D82DE528B40408E56C84
:10CDA2006025156C8009741FD3956C401A056C12AE
:10CDB2006D32126B1E7F0B12921212EEB602ED87CB
:08CDC2007D05AF2812E0A2225A
:10E490007BFF7A5379DD752E047F0312E3B175316A
:10E4A000007532997533007534B7126AA6126D7013
:10E4B00012B4BF126D32753104126B217F0B1292B0
:10E4C0001278C9E6701218E66401700C126BAD1276
:09E4D0006AB3126AEF02B4BF2224
:10E2CE0078C9E6FFB402067E017F018029EFB40310
:10E2DE00047F02802178C9E6FFB404067E037F0323
:10E2EE008014EFB405047F04800C78C9E6B40604EC
:10E2FE007F0580027F008F0CE50C78966660081211
:0CE30E00ECDDE478CBF622E478C9F622BE
:10E6F0008F2B126C08126B4EF53B7F0612B4BFE5F0
:10E700002BB4031078C9E6FFB402047F018013EF35
:10E7100004FF800E78C9E6FFB401047F028003EF96
:0EE7200014FF78C9A607126A677F0602B4BF0D
:10EE7D007BFF7A5F79B4752E087F0412E3B17E6053
:0DEE8D007FB512C973126A677F0602B4BF19
:10F03F0078CBE6BF0307FF12DD41A60722FF12DDE3
:04F04F009BA6072253
:10ECBA007BFF7A5979CC752E057F0412E3B1753141
:10ECCA00007532BA7533007534D8126AA6126D709F
:03ECDA0002B4BFC2
:10D41A00752A1EE4FB7D14FF12EB427F0112CE61D6
:10D42A007F0112CE61126D2B12EAA37E327FE512C2
:10D43A00C9737E637F2E12C9737E617FEB12C97333
:10D44A00752E20752F027B0FE4FD7F0312D66B7EAB
:10D45A00637F5312C973126D8712C607126D911238
:10D46A00C607126E0412C607752C13AB747D091217
:10D47A00D48CAB757D0F12D48CAB767D157F0802E8
:0BD48A00C6077F0812C607752C13228E
:10A95D0078C9E6FF700302AA0A08E66032EF24FE0A
:10A96D0060131460192402600302AABB126D3D7BB3
:10A97D00037D098010126D3D7B037D0F8007126DE5
:10A98D003D7B037D157F0812D66BE478CAF62278DD
:10A99D00C8E624FC601214601414601924036003CB
:10A9AD0002AABB126D878008126D918003126E048E
:10A9BD0012C607804378C9E624FE601614601C1485
:10A9CD00602A2403600302AABB126D9B7B037D09E1
:10A9DD008010126D9B7B037D0F8007126D9B7B0397
:10A9ED007D157F0812D66B78CA760122126D3D7BDC
:10A9FD00047D197F0812D66BE478C9F62278C8E673
:10AA0D0014B40700400302AABB90AA1D126DC273B5
:10AA1D0002AA3202AA6C02AA7502AA7D02AA8502B6
:10AA2D00AA9002AAA112DA3F126D8712C607126D03
:10AA3D009112C607752C13AB747D0912AABCAB75A8
:10AA4D007D0F12AABCAB767D157F0812C607E55F98
:10AA5D0054E74408F55F12BA677E637F66804C1237
:10AA6D00E0F57E637F768043752C23126D8A800E10
:10AA7D00752C23126D948006752C23126E0712C649
:10AA8D0007800C126D9B7B017D077F0812D66B78BA
:10AA9D00C9760122E478CBF678C8F608F608F6FBFD
:10AAAD007DFE7F6D12EAA37E327FE512C973227F90
:08AABD000812C607752C1322D4
:107C0E008F2878C9E6FF7003027D6708E660537817
:107C1E00C8E624FA6003027E5BEF24FE6014146053
:107C2E001E240270377A007974127EB9AB747D0906
:107C3E0080257A007975127EB9AB757D0F80187B21
:107C4E00007A007976752DFFE4F52EAD2812D89BBB
:107C5E00752C23AB767D157F0812C60712BA670204
:107C6E00E91178C8E624FD600C14602714603814FE
:107C7E00604F027E5BAD2812D74E752C23126D8A93
:107C8E0012C607E55F5407700512C2F6801612BAC7
:107C9E00678011AD28126E77752C23126D9412C663
:107CAE000712BA6702E9F67B007A007970AD2812E6
:107CBE00DB09752C23126E0712C60712EFE902EDCF
:107CCE0087E528B4031278C9E6FFB404067E017F67
:107CDE00018015EF04FF801078C9E6FFB401067E1F
:107CEE00047F048003EF14FF78C9A60778C9E62441
:107CFE00FE601714603014604924036003027E5B3B
:107D0E00752E23127E8A7D0D8029126D3D7B017D9D
:107D1E00077F0812D66B126D9B127ED6126D3D7BBD
:107D2E00017D13027E21126D3D127ED6126D9B7B5C
:107D3E00017D137F0812D66B126D3D7B047D1902F7
:107D4E007E21752E13127E8A7D137F0812D66B123A
:107D5E006D9B7B047D19027E21E528B4031278C841
:107D6E00E6FFB407067E017F018015EF04FF801049
:107D7E0078C8E6FFB401067E077F078003EF14FF85
:107D8E0078C8A60778C8E614B407004003027E5BE5
:107D9E00907DA5126DC273027DBA027DD4027DE87C
:107DAE00027DFA027E10027E25027E3A126D447B1F
:107DBE00077F09127ECA7B0E7F03127E9F7B0A7D90
:107DCE00017F04027E58126D447B0E7F03127ECA21
:107DDE007F04127E5C7F05027E58126D447F041272
:107DEE007E7C7F05127E5C7F06027E58126D447F7C
:107DFE0005127E7C7F06127E6E7B0A7D017F070256
:107E0E007E58126D447F06127EAB7F07127E6E7B0C
:107E1E00057D017F088033126D447F07127EAB7B98
:107E2E00057F08127E9F127EE002BA67126D447BB8
:107E3E00057D017F0812D66B752E20752F02127EDE
:107E4E00E0126D447B0E7D017F0312D66B227B0AFE
:107E5E007D0112D66B752E10752F027B0A7D0122C5
:107E6E007B0A7D0112D66B752E10752F02227B0AAE
:107E7E007D0112D66B752E20752F0222752F027B77
:107E8E00017D077F0812D66B752E13752F027B01AD
:107E9E00227D0112D66B752E10752F02227B0A7D64
:107EAE000112D66B752E20752F02227B00752DFFC9
:107EBE00E4F52EAD2812D89B752C23227D0112D607
:107ECE006B752E20752F02227B017D0D7F0812D639
:0C7EDE006B227B077D017F0912D66B220E
:10AAC5008F2878C9E6700302ABCE18E624FE6040F5
:10AAD50014606114700302AB6414700302AB881434
:10AAE500700302ABAC2405600302ABCBE528B403CD
:10AAF5000CE566F4700302AC2505668009E5667011
:10AB05000302AC25156685662F126B627F058046AC
:10AB1500E528B4030CE567F4700302AC25056780EE
:10AB250009E567700302AC25156785662F126B6210
:10AB35007F078022E528B4030CE568F4700302ACB6
:10AB45002505688009E568700302AC2515688566EA
:10AB55002F126B627F0912921212C2F602ABCBE57D
:10AB650028B4030CE569F4700302AC250569800976
:10AB7500E569700302AC25156985662F126B627F46
:10AB85000B803DE528B4030CE56AF4700302AC259F
:10AB9500056A8009E56A700302AC25156A85662F8A
:10ABA500126B627F0D8019E528B40309E56BF4602B
:10ABB5006F056B8006E56B6067156B126B5F7F0F2A
:10ABC50012921212D32402EB9078C8E6FF6051E589
:10ABD50028B4030FEFB407047F01801778C8E60493
:10ABE500FF801078C8E6FFB401067E077F07800363
:10ABF500EF14FF78C8A607E4F531F532F53375345F
:10AC0500FC753504753604F5377538017539E77502
:10AC15003A01753B717BDC7A01FDFC7F0612B4BFFE
:01AC2500220C
:10D11A0078C8E67022760108F6F531753238F533AB
:10D12A00753456753502753602126BBD126AB37DB7
:10D13A0098126AF102B4BF78C8E6B40705E478CB5E
:10D14A00F62278C9E66009E4F67E2B7F8E02C9735F
:10D15A0078C9760118E624FE601714601B14601F54
:10D16A001460231460272405702B126B5F7F0580DF
:10D17A0021126B5F7F07801A126B5F7F098013127F
:10D18A006B5F7F0B800C126B5F7F0D8005126B5FEC
:06D19A007F0F1292122229
:10D58300E4FF12EDE77E607FC412C9737E607FF211
:10D5930012C97378C9E670077E2B7F8E02C9737830
:10D5A300C8E624FE601A14602114602814602F1446
:10D5B30060362405703D126CB9126B687F058030AC
:10D5C300126CB9126B687F078026126CB9126B68F4
:10D5D3007F09801C126CB9126B687F0B8012126C6E
:10D5E300B9126B687F0D8008126CB9126B687F0FDC
:04D5F300129212225C
:10E8E00078C8E66404702708E6602378A1E6FE6035
:10E8F00003B4FF08E478C9F608F6800312EBDC786D
:10E90000C9E660037F0022E478CAF67F01227F0215
:01E9100022E4
:10EC4D0078C8E66401701B08E66017EF6483600EF8
:10EC5D0012EBDC78C9E660037F00227F0122E478A5
:05EC6D00C9F67F022240
:10EC720078C8E66401701B08E66017EF6483600ED3
:10EC820012EBDC78C9E660037F00227F0122E47880
:05EC9200C9F67F02221B
:02EBB6008F27A7
:10EBB8007F0278CBE624FD600E14601224037013E4
:10EBC800AF2712E8E0800CAF2712EC4D8005AF2785
:03EBD80012EC72CA
:01EBDB002217
:09F0CB0078CBE6700312F0C222BA
:10E6730078CBE614601B14601B14601B14601B141E
:10E68300601B24FD601C24F96021240F702002EE1E
:10E693004302B13D02BD9102817E029C70E478CBBE
:0FE6A300F622E55F5407700602D11A12A95D2214
:10EF8C0078CBE624FD600A14600A2403700902D2CF
:08EF9C00A602DE4E12E2CE22B5
:10E197008F2778CBE614601D14601F14602114606C
:10E1A7002314602524FD602624F9602D240F702E8A
:10E1B700AF2702D905AF2702B26AAF27028FD0AFC8
:10E1C70027028D81AF2702CD32AF2702F03FE55FEF
:0FE1D7005407700AAF2702AAC5AF27127C0E2289
:10EDC7008F2A78CBE624FD600C14600E2403700FA5
:10EDD700AF2A02D006AF2A02E6B2AF2A12E6F02225
:10E7D80078CBE624FE6018146018146018146018CA
:10E7E80024FD601724F9601C240E701B02E3FC0250
:10E7F800D49502D6DD02E49002ECBAE55F540770C6
:08E808000602D58312D41A2286
:10EFA40078CBE624FD600A14600A2403700902DEAB
:08EFB400A702EE6012EE7D22BF
:10BB78008F2612EBB68F0CE50CB401057526838071
:10BB880007E50C700302BC8878A1E6FF700302BCCD
:10BB980088F4700302BC88E526247D700302BC7516
:10BBA8002481B40800400302BC8890BBB9126DC25E
:10BBB8007302BC6802BC6D02BC6D02BBD102BC72D0
:10BBC80002BC8802BC7802BC80E55F5407600302AF
:10BBD800BC8878A1E6700302BC88F4700302BC88B4
:10BBE8007E327FE512C9737F0112CE617E317F9468
:10BBF80012C973126D0D24BAF582E5F03432126C55
:10BC0800E412C973126DA212EAA378A1E6FF7406C2
:10BC1800D39F50287409C39F402275548012DB6C4F
:10BC280012989978A1E6FF12E84812E1E6BFFC04F1
:10BC380078A176FE12E282BFFC0C80061288DBBF78
:10BC4800FC0478A176FEC216E478CBF67D407F022C
:10BC580012F066126D2B12EAA37E327FE502C973D9
:10BC6800C21602E673AF2602E19702DC8B02E7D820
:10BC780078CBE6700B02F053E56F30E30312F0CB9C
:01BC88002299
:10EBDC008F29E52924FD601214600F24FE60102497
:10EBEC0083600F2481700E02EF8CAF2902EDC712E7
:06EBFC00DC8B12EFA422E5
:10D9D700E4F531F532753301753408126B4F753B39
:10D9E700017BE87A01FDFC7F0712B4BF7F8012F04C
:10D9F7002A7E327FCE12D50E126DA212EAA3E478E8
:10DA0700A6F608F678A6E6FE08E6FFC39470EE646D
:10DA17008094805014126B29753B017F0712B4BFA5
:10DA270078A77406126D0680DB78A7126DCD126B8E
:08DA37003AF53B7F0702B4BF82
:10E31A0078A6760008767078A6E6FE08E6FFD3941B
:10E32A0000EE648094804018126B29753B017F07C8
:10E33A0012B4BF78A774FA26F61874FF36F680D797
:10E34A00126D2B12EAA37E327FE512C97378A712E7
:0CE35A006DCD126B3AF53B7F0702B4BF9B
:10DFA8007D407F0212F066126D2B12EAA37F0112E8
:10DFB800CE61E55F540714601614601914601C14D0
:10DFC800601F146022240570257E2F7FEE801C7E42
:10DFD800307F4880167E327FCA80107E327FCB80A9
:10DFE8000A7E327FCC80047E327FCD12C973126DD7
:04DFF800A202EAA3F4
:10D5F70078A1E670417D407F0212F066126D2B1212
:10D60700EAA3E55F54077014900F3BE030E00D127A
:10D617006D0D2486F582E5F0346380127E637F2EDC
:10D6270012C973126D0D2496F582E5F03463126CFE
:10D63700E412C973802778A1E6F460033008247DDB
:10D64700407F0212F066126D2B12EAA3126D0D24B1
:10D65700A6F582E5F03463126CE412C973126DA269
:04D6670012EAA322FE
:10C2A80001940002A200000292000002980000021D
:10C2B8009B0000019700C10DC10BC10CC10AC10947
:10C2C800C10801A40001A00001A100019A00019E7B
:0AC2D80000019600019F00019D0087
:1079040078A1E675F00AA42417F582E5F03405F5AC
:1079140083E493FE7401932278A2A905AA06AB0717
:10792400E6FE08E6FFE4FCFD2275F00CEEA4244913
:10793400F582E5F03402F5837892E6FC08D3E6FD9F
:107944007401939DE4939C22EF2BFFEE3AFEED39F4
:10795400FDEC38FC780612887E8F1B8E1A8D198CEC
:107964001822F9F812873DA804A905AA06AB072234
:10797400E4FCFD7B64FAF9F802873D75F00AE5281A
:10798400A42419F582E5F034052212873D8F0F8E69
:107994000E8D0D8C0CAB0FAA0EA90DA80CE4FFFEE6
:1079A4007DEE7C021287C87897EFF622E52875F001
:1079B4000AA424AEF582E5F03407227886E6FE08B0
:1079C400E6FBAA06E4F9F8227893E624FFFF18E61A
:1079D40034FF221287C88E298F2AE529C313FEE5B6
:1079E4002A13FF7C00E52A54012FF52AEC3EF529E1
:1079F4002285111353120F850F11531087850D0F14
:107A0400530E8F227891A6077890E6FF7880E6FDE2
:107A1400FB7A002FFFE433FED374809FE49E22F5AB
:107A240083E493FC740193221287C88E0C8F0D2279
:107A340018367893FEE6247EFD18E436CDC39F22E3
:107A44007886E6FE08E6FFC322FB7A04F9F802878B
:107A54003D7801AF1BAE1AAD19AC1802886B78A241
:107A6400E6FE08E6FF2278A1E675F00AA422E4F512
:107A74000D750E067884E6F50F18E6F51022AE298A
:107A8400AF2AAB07AA06E4F9F822FF7A687926E45C
:107A9400FCFDFBF802873D75F00CEEA42445F5824D
:107AA400E5F03402F58378A2227892E6FC08E6FD3C
:107AB400D322FF24FFFDEE34FFFCE6FA08E6FBC305
:107AC4009DEA9C2278A1E614131313541F7894F6AC
:107AD400FD7B017FAE227C001286D678A2E6FC08EC
:107AE400E6FD2275F00CEEA4244BF582E5F0340299
:107AF400F583C3227883A60608A60722C3E52A785D
:107B04008796E52918962275F00CEEA42447F58291
:107B1400E5F03402F583227892E6FE08E6FF227847
:107B240091E62BFFE43AFEC3747E9F74019E227893
:107B3400A2A60E08A60F7892A61008A61122791004
:107B4400FBFAF802873DAE2BAF2CE4FCFD02873D27
:107B5400E50C788426FFE41836CF22C3748A950D89
:107B6400E4950C22E62401FFE433A2E713EF13FFAC
:107B740022ED2402FBE43CFAC3EB9FEA9E22EF24AD
:107B840003FFE43EFED3EB9FEA9E227BF4F97A01E5
:107B9400F802873D750C05E4F50D22748AC3950F30
:107BA400E4950E2278A1E6FF75F00A227A60FBF9CB
:107BB400F802873DE624FE18E634FF22E50CA2E332
:107BC400920CA2E2920A22D3E528942DE527940090
:107BD40022A4241BF582E5F0340522750C07E4F594
:107BE4000D22E51B5401FFE4FEFDFC22750C0EE49E
:107BF400F50D750E75227989E7788726FF19E72236
:0A7C0400C3747E7880967991F72210
:10E76700E55F540714600304701BA20A920BA20C06
:10E77700920D78A1E6FF6003B4FF05128B2E801679
:10E7870012C150801178A1E6FF6003B4FF0512F0B3
:09E79700FD800312F10602EE06FA
:10EE0600E55F540714601004700D78A4E670047D65
:0FEE16000280067D3280027D027F4C12F0662260
:10DF5300EF14600E14601414601A240370207D0102
:10DF630080027D037F4A12F066801312DF9C7A07DA
:10DF73007984800712DF9C7A07798512E446E55F8E
:10DF83005407700978A4E660047D3280027D027F25
:10DF93004C12F0667F2302F02A7BFF7A07798812FE
:05DFA300E4467BFF22B3
:04A7F1008E278F28F8
:10A7F5007D0C127ADA1286E88F0C7FFF7E2C127A96
:10A805009BE6FC08C3127942400302A90E127B0B9A
:10A81500D3127944500302A90E12792D400302A9DF
:10A825000E127AE7127944500302A90EBE2C0EA22D
:10A835000A720C500302A90C7E2B02A90CBE200E35
:10A84500A20A720C500302A90C7E1F02A90CEE6429
:10A855000E702AA20C300A01B35022300A0FE50C03
:10A8650060047D0380027D43AE0502A90CE55E30E0
:10A87500E4047D0480027D44AE0502A90CEE640D5E
:10A885007028A20C300A01B35020300A0EE50C6086
:10A89500047D0180027D41AE05806CE55E30E404F7
:10A8A5007D0280027D42AE05805DBE0C13300A0735
:10A8B500200C047E0A8050E55E30E44B7E0B804719
:10A8C500EE6409701D300A11200C0EE50C60047D44
:10A8D5000680027D07AE05802EE55E20E4297E0810
:10A8E5008025BE1B09127BCB401D7E1A8019BE1A1E
:10A8F50009127BCB50117E1B800DBE1E0A7897E690
:10A90500D3944750027E1DAF061EEE6007EFF4702C
:10A915000302A803EFF4703F7886F608F67E3A1234
:10A92500792D5028127AE71279444020EE1279B237
:10A93500127A237886A60408F6127A9B12793E507D
:10A945000B127B0BC31279444002AF061E7433D33E
:07A955009E5004EFF460C8FE
:01A95C0022D8
:10AEC900127A44E49F74049E400302AF53127974CA
:10AED900C00412791CD00012873DC004C005C00609
:10AEE900C007900777127915127A8ED003D002D055
:10AEF90001D000127A2C127B5F504C1279CCFE12D1
:10AF09007974C00412791CD00012873DC004C005B1
:10AF1900C006C007900777127915FFE4FCFD7BA0F6
:10AF29007927127B92D003D002D001D0001287C8B2
:10AF39008E0E8F0F127B9F50097886760408760053
:10AF490080087529BD800375293D127A44E49F74F0
:10AF5900049E500302B006127974C00412791CD001
:10AF69000012873DC004C005C006C00790076D12D6
:10AF79007915127A8ED003D002D001D000127A2C22
:10AF8900127B5F50751279CCFEC374109F74049EB6
:10AF99004027127974C00412791CD00012873DC071
:10AFA90004C005C006C00790076D127915FFE4FCBF
:10AFB900FD7BA07A017927801F78A2127924127962
:10AFC90077C004C005C006C00790076D127915FF48
:10AFD900E4FCFD7B9A7A09F9F812873DD003D00287
:10AFE900D001D0001287C88E0E8F0F127B9F50059B
:0FAFF9007529FF80087529BC800375293CAF2995
:01B008002225
:10E6330078A1E6703278A4E6B4100C7E0A7F9812B3
:10E64300E66BE478A4F62278A4E6700C7E0A7FB821
:10E6530012E66B78A47620227E0A7FAA12D50ED208
:10E663000CD20A78A476102212D50ED20CD20A222A
:01F1050022E7
:108B2E00E4FB7D097F4C12ED44E50C30E114E55F6A
:108B3E00540770047D2080027D007F4C12F0660287
:108B4E008C43127A627898A60608A607127B1B78C9
:108B5E009BA60608A607127BC01279F5127B33E599
:108B6E005F5407700685122585132678A212792484
:108B7E00C00412796D127B1BE4D00012798E30E0A6
:108B8E0005127B6880067897E6C313FF7897A607D1
:108B9E00127A627898127AAF9FEC9E500C127B7507
:108BAE00400778A2A60408A605127B1B789B127AB2
:108BBE00AF9FEC9E500C127B7540077892A604086E
:108BCE00A605A20C300D01B34008A20A300B01B36A
:108BDE0050447B017D017F0512ED44E55F5407FF94
:108BEE007019530CD7200A03430C20200C0878A4CC
:108BFE00E67003430C087524FF8012BF010F530C5F
:108C0E00F3200C03430C08200A03430C04AD0C7F25
:108C1E000512F0668074127A62D374FF9F74079EF9
:108C2E004013127AAD74FF9D74079C4008EF4E609E
:108C3E0004ED4C7005E4F5248050E55F540770098F
:108C4E00AF26AE2512A7F180027FFF8F247897E61C
:108C5E00FF7430D39F5006744CC39F50057524FF8C
:108C6E008028E524B4FF147887E61846600DE55F8A
:108C7E005407700712AEC98F24800FE55F5407FFAB
:108C8E00BF0107AF2412A18E8F24E55F5407FB703E
:108C9E001978A4E6B42013AE25AF267D07127ADA32
:108CAE001286E8EF4E6003E4F524E524F46004E553
:108CBE00247069EB700978A4E6B42003E4F52478F7
:108CCE009AE6FFF46007EF6004E4789EF6789AA6C1
:108CDE00247405D3789E96401306E55F540764010D
:108CEE006003028D807D037FFF02F066E55F54070F
:108CFE00FFBF0107E4FD7FFF12F066789AE6FF786A
:108D0E00A1E6B50703D38001C3920978A1A607781F
:108D1E009E7603E55F5407705902E633789AE6654E
:108D2E00246011789E7601789AA624E55F54077028
:108D3E004102F105E55F54077F038F0CE50CD378F4
:108D4E009E9640020622900F317401F07D407F0204
:108D5E0012F0667E327FE512C973789AE678A1F634
:108D6E00E4789EF6C209E55F540770030275B612E9
:028D7E0083FF71
:018D800022D0
:10C15000E4FB7D057F4C12ED44E50C30E110E55F1A
:10C16000540770047D2080027D007F4C8055127B37
:10C17000C01279FB127B33A20C300D01B34008A230
:10C180000A300B01B350417B017D017F0512ED4464
:10C19000E55F5407FF7016530CD7200A03430C20A9
:10C1A000200C1C78A4E67017430C088012BF010F06
:10C1B000530CF3200C03430C08200A03430C04AD7A
:10C1C0000C7F0512F0668045127A62D374FF9F746B
:10C1D000079E4013127AAD74FF9D74079C4008EFD0
:10C1E0004E6004ED4C700280247898E6FE08E678F4
:10C1F000A2127AB64017127B825012789BE6FE0894
:10C20000E67892127AB64005127B824006789A76DA
:10C21000FF800678A1E6789AF6789AE6B4FF0302E2
:05C22000BE95D20922C9
:02A18E008F2719
:10A190007D037F4C12F06675283C7F0112F02AE4A3
:10A1A000FB7D077F4C12ED44E50C30E103D528EA36
:10A1B0001279F5E50F450E6020D374FF950F7407F3
:10A1C000950E4015E5114510600FD374FF9511747D
:10A1D0000795104004E528700AE4FD7F4C12F066F4
:10A1E0007FFF22E50F25E0797BF7E50E3319F7783D
:10A1F00086A61008A611E51325E07982F7E512334B
:10A2000019F7D3745E95117401951040037FFF22F6
:10A210007881E6FE08E6FF5407FDC374029DE494CE
:10A2200000500AEF2408FFE43EFEEF80067881E646
:10A23000FE08E654F8FF7881EEF608EFF6C3E49FD7
:10A2400074059E50061876050876001279CCFEE457
:10A25000FCFD127A4DE47B107A04F9F8127A2CC3D3
:10A26000E50D788796E50C18965005A60C08A60D06
:10A2700075273CE527643C600302A333752833123D
:10A2800079B0127913FF12797F127A23FDC39FEC04
:10A290009E502A7886E6FE08E6FFED9FEC9E40037E
:10A2A00002A3221279B0F5837401932418FDE4937C
:10A2B0003400FCC3ED9FEC9E501402A32212797F60
:10A2C000F583127A447401939FE4939E405475F091
:10A2D0000AE528A42415F582E5F03405127913FF68
:10A2E000E4FCFD7B9A7A0912796612797F12791360
:10A2F000FF127B4EC004C005C006C00778861279E5
:10A3000024127977C00412791CD000127968D00722
:10A31000D006D005D004127A2CD3127B604003AF54
:10A3200028220528743BC39528400302A27F12AE61
:05A33000C98F27AF27D3
:01A335002205
:03F0FD0002F1001D
:01F1060022E6
:10C6C0008F2B8D2C8A2D8B2EEFFD7C00788926FBFD
:10C6D000EC1836FAE52EAE2D7806CEC313CE13D85D
:10C6E000F9FFC3EB9FEA9E501BC3EF9D7889F6EEDE
:10C6F0009C18F608E6FD7F0A12F0667888E6FD7F52
:10C700000B12F066E52C75F040A4FFAEF07C007DC6
:10C710000A1286E8AC06AD07E52B788926FFE418F7
:10C7200036FEEF7806C333CE33CED8F92DFFEC3E7C
:10C73000CFC3952EF50DEF952DF50CE50DAE0C78CC
:10C7400006CEC313CE13D8F97880F6E6C43333543B
:10C75000C0FFC3E50D9FF512787A1279C1AF12FCC4
:10C76000FDFE12873DE4FB7A04F9F81287C88F12A8
:07C77000AD127F1E02F0660E
:109AA3008E2B8F2C127BA8127BD5F58374019370B8
:109AB30002E4936024750C06E4F50D750ED0750F62
:109AC3001175F00AEF127BD5127A23FDECF5108D98
:109AD30011E4F5127F0C02E4D9788A1279247B8091
:109AE300FA127966127B4AC004C005C006C0077823
:109AF30086127924C00412796D127A62E4D00012BE
:109B03007968D007D006D005D004127A2CE50D78F9
:109B130002CEC313CE13D8F9F51BFF7E007C007D64
:109B2300281286D67DB01286E8EF24FBF511E4F502
:109B330012E511D3943C400974C42511F511431265
:109B430080E511D39428400974D82511F5114312E7
:109B530040E511D39414400974EC2511F511431217
:109B630020E511D3940A400974F62511F511431227
:109B730010E511D39405400974FB2511F511431227
:109B830008127BDF750ED085120FE51B24FEF5103E
:109B930075111E751204E4F5137F0C12E4D91279C2
:109BA300BFFFFE7D777C011287C812796B127B4A57
:109BB300C006C00778A21279C1D007D0061287C8A1
:109BC300C004788A12791ED00012873D8F0F8E0E43
:109BD3008D0D8C0CE51B2401FFE433FE7A8079BBE9
:109BE300127A93E47B10FAF9F81287C88F138E1256
:109BF3008D118C10C3E513950FF517E512950EF52E
:109C030016E511950DF515E510950CF514780F1261
:109C1300886B12795DAF17AE16AD15AC14780112CF
:109C2300887EAB1BAA1AA919A8181287C8EFF51BBF
:109C3300EE540FF51AE4F519F518AD1B7F9A12F0DF
:109C4300667808127A57EF4420FB7DF07F9B12EA77
:109C5300A37B087DFF7F5A12EAA37B207DFF7FD27F
:0D9C630012EAA3E4FB7D7F7FD312EAA32267
:1064560078A1E6FF54C0F528EF543FF67B027DF99C
:106466007F7012EAA3E55F5407FFBF011CE4FB7DC2
:10647600F97F7012EAA3127A6A24A8F582E5F0344D
:10648600071279137883026627E52830E6299008F3
:1064960000127915FF787AA60608A6079008021258
:1064A6007915FF127AF8900804127915FF7881A6FB
:1064B6000608A60702657D127BA8A424A6F582E538
:1064C600F03407127A23787AA60408F675F00AEFF4
:1064D600A424A8F582E5F034071279137883A6067A
:1064E60008F6127A6A24AAF582E5F03407127913BF
:1064F6007881A60608F678A2127924127B8FC0044A
:10650600C005C006C007787A127924127BB0D00382
:10651600D002D001D0001279D7C3748C952AE495A5
:1065260029505478A1E6FF74379F504B743BC39FA4
:106536004045E6FF75F006A424C8F582E5F0340868
:10654600127A23787AA60408F675F006EFA424CA10
:10655600F582E5F034081279137883A60608F678F2
:10656600A1E675F006A424CCF582E5F0340812798C
:10657600137881A60608F678A2127924127B8FC0BA
:1065860004C005C006C007787A127924127BB0D001
:1065960003D002D001D0001279D7D3742D952AE406
:1065A600952940047B1580027B057DE07FEA12EA8F
:1065B600A3D3743C952AE4952940047B0880027B8A
:1065C600007DF37F0412EAA3E4FD7F3C12F0667DB2
:1065D600067FEB12F0667B407DFF7FEC12EAA37D1F
:1065E6001D7FE812F066E4FB7DC77FEB12EAA37B12
:1065F600047DFF7FFF12EAA378A1E6C3941D500431
:106606007D0880027D107FE912F06678A1E6FF74AE
:106616003CD39F401075F00AEF1279B512791378C2
:1066260086A60608F67D037F8C12F066127A6A2427
:10663600ACF582E5F03407F58374019324FC788980
:10664600F6E49334FF18F67D067F8D12F06678A186
:10665600E6FFC394175005750C02800EEFC3942C09
:106666005005750C058003750C03127B5424FA083B
:10667600F6EF34FF18F6127BA8127984F583E493BB
:10668600F529740193F52AEF643C701FE52830E77D
:10669600481279CCFED374109F74049E7886E64027
:1066A600028016F52908E6F52A802E78A1E6B43D83
:1066B60028E52830E7237886E61279257B10127ABA
:1066C6004EC006C0071279CCAB07FAE4F9F8D0073A
:1066D600D0061287C88E298F2A78A1E675F00A128D
:1066E6007984127913FFC3952AEE952950048E29D1
:1066F6008F2A127B004012127904FFC3788296EE2D
:1067060018965005A60608A607D3127B0140034338
:106716002801127B005003432802127904FF788176
:10672600127AAFEF9DEE9C4003432804C3EF9DEE23
:106736009C5003432808750C0B127A727882E6F592
:1067460011ECF5127889E6F51318E6F5147887E664
:10675600F51518E6F516E4F5177F0C12E4D9127B49
:10676600DF750E40E52830E30A127904F50FEEF5E1
:1067760010800685110F851210E52830E109852A5B
:1067860011E529F5128006851511851612E4F51313
:106796007F0C12E4D9E528540A60067B017DFF8050
:1067A60004E4FB7DFE7F7012EAA3E52830E0067B59
:1067B600027DFF8004E4FB7DFD7F1512EAA3E52838
:1067C60030E2067B017DFF8004E4FB7DFE7F15122F
:1067D600EAA3127BDF750E71E52830E33378811268
:1067E6007924127B42C006C0071279041279C5D0FB
:1067F60007D0061287C812795D780812886BEF24D5
:1068060002F511E43EF51085110F7B407DFF8009EE
:10681600E4F50F751010FB7DBF7F0412EAA3E5288F
:1068260030E1377886127924127B42C006C00712FF
:106836007A82D007D0061287C812795D7808128846
:106846006B8E128F13E51B7008E513151370021576
:10685600128513117B807DFF8009E4F511751210F6
:10686600FB7D7F7F0412EAA3E4F5137F0C12E4D9C3
:10687600750C08E4F50D750E16E52830E2427881B0
:106886001279247908127B44C006C00712790412D3
:1068960079C5D007D0061287C812795D127BE6C08B
:1068A60004C005C006C007127A55D003D002D00135
:1068B600D00012794C851A0F851910851B13800993
:1068C600750FFF7510FFE4F513E52830E04678866E
:1068D600127924FBFA7908F812873DC006C0071220
:1068E6007A82D007D0061287C812795D127BE6C07D
:1068F60004C005C006C007127A55D003D002D001E5
:10690600D00012794C851A11851912E51BC4540F53
:10691600421380067511FF7512FFE4F5147F0C1201
:10692600E4D97D2C7F2012F066127B98750E291211
:106936007A6A2417F582E5F03405F5837401932409
:1069460020F511E4933400F51085110F751105E457
:10695600F512751334E52A240CF517E43529F516D6
:10696600851714F515E4F5167F0C12E4D9127A6A28
:106976002415F582E5F03405127913788AA60608FF
:10698600F6200E047D2D80027D2F7F2012F066AF4B
:106996002AAE29129AA3127B98750E22788BE624CA
:1069A600FEF50F127BB8126A5CE52820E00330E1A1
:1069B600227892127924127A4DC006C0071279BF46
:1069C600D007D0061287C8EF2440788FF6E43E1829
:1069D600F6800D7893E62440798FF718E43619F798
:1069E600127B98750E2D788FE6F50F18E654071270
:1069F6006A5C78861279247A03127BB2C006C007D5
:106A0600127A82D007D006127A2CE52830E008AB3D
:106A16000DAA0C7D05800BE528AB0DAA0C30E1060E
:106A26007D067F0280047D097F0112C6C0E4FB7DDE
:106A3600FC7F6812EAA37880E6FD7F3812F066E4F0
:106A4600FD7F0112F066E4FD7F1F12F0667B017D7B
:066A5600FF7F0402EAA329
:0B6A5C00F510E4F5117F0C12E4D922C4
:1075B60012645612DCE77882E6B4001318E6B405C6
:1075C6000EE560B402097B017DFF7F1512EAA31266
:1075D600F01512F0F712E56A12F07912BA6778A17F
:1075E600E6FF12EB1BE4789FF6741CD39554500704
:1075F60074E4C3955450037554801298997F06120B
:10760600F02A789DE670257FCA1278F17D0D7FCA33
:1076160012F0667F0412F02A7FCE1278F1E50C751F
:10762600F0C8A4E5F078BEF6789DA60C78BDE670A5
:107636000312CC97129899788D76B2788C764E781C
:10764600A1E614FD7B017FAE12E5F1E50CD394E4CF
:107656004003E4F50CE50C30E71A2480FFE434FF20
:10766600FE7884E624CEFD18E634FFCDC39FFFEDF9
:107676009EFE8009127B5424CECF34FFFE127AF888
:10768600127B98750E06127A7AE4F5117F0C12E4D5
:10769600D9788DE6FFC3955250048F52800B788CB3
:1076A600E6FFD3955240028F5212DB6C53557CAFE6
:1076B6005512B94A7D011278F9E4FD1278F9127B68
:1076C600F0F50F7510FF751107F512F513F514F5A2
:1076D60015F516F517F518751901F51A7F0C12E44C
:1076E600D975273C7F0112F02A7B017D017F7F122D
:1076F600ED44E50C30E003D527EAE4FD7F7F12F088
:1077060066E527602AE4FB7D047F8012ED44E50FE1
:10771600540FF50C850E0D7892127A46950DEE955E
:107726000C500AAC0CAD0DAE04AF058005800312FB
:107736007B1B78B7A60608A60778A1E6FF7433D3A5
:107746009F504D75F00CEFA42449F582E5F0340204
:10775600127913FFC378B8E69FF50D18E69EF50C6F
:107766007880E6FF7E00250DFDEE350CFCC374FE29
:107776009DE49C500AC374FE9FF50DE49EF50C78BB
:1077860089E50D26F618E50C36F67880E50D26F621
:107796007888127A4674809FE49E50067C007F00AB
:1077A6008005C374819FFF7890EFF6744ED39F4097
:1077B60002764E127BFA183678B8127A38F50DED45
:1077C6009EF50CD3E50D94FFE50C940040047FFF75
:1077D6008002AF0D127A08400674809D7890F612EA
:1077E6007B235003127C0474B2C3789196500276C0
:1077F600B27890E6FFD3955340048F538019C3E4C3
:107806009FFF74019400FEC3EF9553EE940050075A
:107816007890E6F404F55312C77778A2127924C05B
:107826000412796D78B7E6FE08E6FFE4D000127917
:107836008E30E005127B6880067897E6C313FF78E2
:1078460097EFF6D3944E4002D208127ADF7E607F1D
:10785600001286E8D3EF945AEE94004002D2081242
:107866009E2A8F0CE50CB4010A7F0A12F02A129E9A
:107876002A8F0CE50C6003C38001D39212E478BF13
:10788600F6FB1278E27B401278E27B807D3F7F6DCB
:1078960012EAA3E4FD7F6C12F0667B207D7F7F20D9
:1078A60012EAA33012097B207DDF7F8E12EAA31233
:1078B6007AC812E5F17894E675F008A4FFC378A1BA
:1078C600E69F7894F614FFE50CA807088002C31318
:0B78D600D8FC7894F65401F6436520BE
:1078E100227D3F7F6D12EAA3E4FD7F6C12F06622D8
:1078F1007B017D0112ED44227F7F12F0667F281209
:03790100F02A2247
:1083FF001264567888127A4674809FE49E50067CE9
:10840F00007F008005C374819FFF7890A607127BC1
:10841F00FA127A34F515ED9EF514C374FF9515E431
:10842F00951450047FFF8002AF15127A084006742E
:10843F00809D7890F6127B235003127C0478A1E67E
:10844F00FF12EB1B12E56A12F07912BA6712DCE722
:10845F00127BF0750F02787BE624FEF510127BB8C5
:10846F00F5117512027893E624FEF513127BB8F519
:10847F0014E4F515F516F517F518751981F51A7F2A
:10848F000C12E4D975273C7F0112F02A7F7F1286E8
:10849F007430E003D527F0E5277009FD7F7F12F0D8
:1084AF006602BE95E4FB7D087F8012ED44E511FE68
:1084BF007C00E42510FFEC3ECF24FE7884F6EF34E9
:1084CF00FF18F6E50DFEE4250CFFEC3ECF24FFF57B
:1084DF000DEF34FFF50C7891E6F9FF7888E6FC088C
:1084EF00E6FD2FFFE43CCF2480CF34FFFED3E50D14
:1084FF009FE50C9E50030285A0ED788726FFEC12B6
:10850F007A34F50FED9EF50E7880E6FF7891E6FE52
:10851F002F24807880F6EEFF7E00788926FDEE18F6
:10852F0036CD248008F6ED34FF18F6C3EF950FEE25
:10853F00950E4003028606E9FFC3E50F9FFFE50E88
:10854F009EFEC3E50D0896FDE50C1896FCC3EF9D46
:10855F00EE9C400BED2403F50FE43CF50E801F78E5
:10856F0089E6250FFF18E6350EFE7891E6FDC3EF7D
:10857F009DFFEE9400CF2403F50FE43FF50E747EBC
:10858F00127BA15006750E00750F7EE50F4480809B
:10859F00477890E67889127B582480CF34FFFEC34A
:1085AF00E50D9FE50C9E50387880E6789026248064
:1085BF007880F67888EEF608EFF6C3950DF50FEE96
:1085CF00950CF50ED37403950FE4950E5003E480CC
:1085DF0007C37403950F4480FD7F8C12F0668017DC
:1085EF00E50D788026FF7889E6FEC3EF9E7880F64A
:1085FF007888A60C08A60D7FFF1286745403600BB3
:10860F00788474F226F61874FF36F6750C05127A14
:10861F0072751105E4F51275130A7889E6F51418C9
:10862F00E6F5157516047517017518387880E6F597
:10863F0019E4F51A7F0C12E4D97F0812DBCC129ED5
:10864F002A8F0CE50CB40105129E2A8F0CE50C60E5
:10865F0003C38001D39212E478BFF67B207D7F7F26
:04866F002012EAA348
:0B867300227B017D0112ED44E50C228A
:01F1070022E5
:03F1000002F10712
:10EA4E007B017D017F4C12ED44E50C20E104E4785E
:10EA5E0095F67895E6600216227895760212B5E75D
:0BEA6E00200907D2147F0212EA79226F
:10C4860020090302C53520120302C535E56520E5FE
:10C496000302C53578A1E6700302C535F4700302C0
:10C4A600C5357894E6700302C5357F0112CE617FEB
:10C4B6000112CE6112C5367B017DFE7F6D12EAA3A5
:10C4C6007E317F9412C973E55E540775F002A42489
:10C4D600BAF582E5F03432127913FF12C973128865
:10C4E600DB12C5365365DF12E96E127AC812E5F122
:10C4F600750D017894E6FF75F008A4FE78A1E614A0
:10C50600C39EFEE50DA806088002C333D8FCF50DD0
:10C51600F4550CF50F750C04750DAE8F0E7B007A75
:10C5260000790C12E4467F1012F02AE47894F62281
:10C53600E4FB7DFE7F6D12EAA37E327FE512C973AE
:01C5460022D2
:04C2E200C10FC10EB9
:10F015007DF27FD612F0667D407FDA12F0667D4084
:05F025007FE602F06629
:10EEEE007DF37FD612F0667D417FDA12F0667D47A4
:0CEEFE007FE612F0667D5F7FDD02F066AB
:07F0D4007D0F7FA002F06632
:07F0DB007D8F7FA002F066AB
:01F1080022E4
:01F1090022E3
:07F0E2007E0A7FCB02D50E70
:07F0E9007E0A7FC602D50E6E
:10BF8400EF700302C02612F0E97F0A12F02A12C0F1
:10BF94004CE4900F30F0D20E7F2812F02A7D0C7FF3
:10BFA4002112F0667B037DFF7F2012EAA37B207DB4
:10BFB400FF7F3A12EAA3E4FB7DDF7F3A12EAA37E15
:10BFC400227F317BA17A00E4FDFC12C070E55E544F
:10BFD40007FFBF070C7E0E7F1D7B4B7A007D7380AD
:10BFE4000A7E147F087B457A007DA97C0512C07007
:10BFF4007E1A7FFD7B707A007D287C0812C0707EDB
:10C004002A7FE57B067A007D0A7C0212C070E4FD7B
:10C014007F0112F066E4FD7F1F12F066E4900F3199
:10C02400F022900F317401F07F7812F02A7E327F73
:10C03400E512C97312C04C900F307401F0C20E7F28
:10C044002812F02A12F0E222E4FD7F2112F0667B2E
:10C05400017DFD7F2012EAA37F1412F02AE4FB7D08
:0CC06400FE7F2012EAA37F1412F02A22B3
:10CEEE008F24200F2DE5246480707BD20F12E14732
:10CEFE0012F104C209D214C2127895760212EE060D
:10CF0E00E4FF12EA79535EF712E96E7F0A12F02AF5
:10CF1E008054E52464817052435E0812E96E7F0AE4
:10CF2E0012F02AC20FE4FF12BF84C21912EF257D40
:10CF3E00427F0212F0667BFF7A07798712E446126F
:10CF4E00F01512F10812F0D47FFA12F02A7FFA12BD
:10CF5E00F02A7FFA12F02A7FFA12F02A7FFA12F0E4
:0CCF6E002A7F0312EA79C210D322C322EA
:08C2E600C117011F00011E0039
:08000300E4781EF608E6FF2276
:10E8AE00E55F5407FF7896E6FE6F6024EE5407FF8F
:10E8BE00E55F54F84FF55F12E96E7895760212BE59
:10E8CE009512AD7812EE067F0112EA79C210D322AC
:02E8DE00C32253
:10ECDD007401C39F401CEF70028014BF010578962C
:10ECED00760122EF64026003BF0303E48001E47840
:03ECFD0096F62266
:10B5E700E55F5407F50C600964016005E50CB403D9
:10B5F70002B21720170312E76720090302B70A20D0
:10B60700170302B70A781FE6FF12DF53781FE660B9
:10B61700076401600302B6ADE4FB7D097F4C12EDC0
:10B6270044E50C30E10D7D207F4C12F066750E80ED
:10B63700751080E51020E757E50E20E752850F11BA
:10B64700531087850D0F530E8FC3E50E94045028B2
:10B65700E50F9404E50E9401401EE51194ECE51006
:10B6670094045014E51194AEE5109401400A781E35
:10B67700E69403504A06806E12000370067E017F2F
:10B6870001805FEFB401047F0380027F00805312C3
:10B69700000370067E017F01800AEFB401047F0377
:10B6A70080027F00803C7B017D1F7F4212E5F1E530
:10B6B7000C20E619781EE6C394035003068027780A
:10B6C7001FE67896F6E4781FF618F680191200033D
:10B6D70070067E017F01800AEFB401047F038002B8
:10B6E7007F00781FA607E4FD7F4A12F066E55F54E6
:10B6F70007700978A4E660047D3280027D027F4CE2
:04B7070012F06622B4
:07C2EE00C110C11101D000D5
:03000B0002EC0202
:10EC0200C0E0C0D075D000C000758AFF758C5FD29D
:10EC12001078C5E61846600708E61618700116D087
:06EC220000D0D0D0E0326A
:03001B0002EE25CD
:10EE2500C0D075D000C007C28E758BFF3013047F2C
:0EEE3500FB80027FF78F8DD211D007D0D03234
:10F02A00EF6011C211D28E3011FDC2111FEF6004C0
:05F03A00D28E80F322DC
:10C82200A2E19290D294C294A2E29290D294C29443
:10C83200A2E39290D294C294A2E49290D294C2942F
:10C84200A2E59290D294C294A2E69290D294C2941B
:10C85200339290D294C29422D294C294A29022850E
:10C862003082852F832293FFE4FD12EF5F7402254D
:10C8720031F531E43530F53022929712ED66D296D9
:10C8820012ED66C29622350AF583E493F50975081E
:10C8920080050BE50B22E509550824FF9218E508EF
:10C8A200C313F5082212F0F0C2950B7F9202EF5FDC
:10C8B200C295E4FBFD7F9002EF5F0530E530AE2FBD
:0AC8C2002274019324FCFF02F0072A
:10ED6600000000000000000000000000000000009D
:10ED7600000000000000000000000000000000008D
:01ED8600226A
:04E5F1008F298B2AB9
:10E5F500E52A6039E4FB12EF3F7B01E4FDAF291208
:10E60500EF3F152AE4F52BE52BC3952A5010E4FFBF
:10E6150012EACC740C252BF8A607052B80E97F019F
:0DE6250012EACC740C252AF8A60712F09B0F
:01E6320022C5
:06E446008B328A33893499
:10E44C0012867EFF7403D39F50398F3690000112D1
:10E45C008697FF900002128697FDE4FB12EF3F7542
:10E46C003503E535C395365017AB32AA33A934853D
:10E47C003582758300128697FF12EFBC053580E25A
:03E48C0012F09BF0
:01E48F00226A
:10EACC00E4FEFDD29612ED66EE25E0FEA297E4334D
:10EADC004EFEC29612ED660DBD08E8EF1312C87B10
:07EAEC0012ED66D297AF06A0
:01EAF3002200
:10EFBC00E4FEEF3312C87BEF25E0FF0EBE08F3D260
:07EFCC009712C88002ED66F8
:10EF3F00AE07D296C29712ED66C296EE2BFF12EF76
:0AEF4F00BCEB7005AF0512EFBC2209
:0FF09B00C29712ED66D29612ED66D29702ED661D
:10E9C90012C85A920012C85A920112C85A920212D7
:10E9D900C85A920312C85A920412C85A920512C808
:0DE9E9005A920612C85A9207D294AF20220B
:08EFFF0014F5828E83E493FFF8
:0EF00700EF1312C853EF12C822D290D29422F7
:06EF590004F8E6FFE4FDF0
:10EF5F0012F007D290D294ED1312C853EB1312C8CC
:04EF6F0053D29022C7
:07F0F000C294D294D29522D4
:10ED4400AE07AC05EC601AC2957D0112EF5FE4FEDC
:10ED540012E9C9AD060E740C2DF8A607DCF212F008
:02ED6400F0229B
:02E4D900AE078C
:10E4DB00A806E6FF54FC603EEF24FDFC0EC295A897
:10E4EB0006E6FA64027016E87B0112EF590E0EA8CD
:10E4FB0006E6FDAF0512F007DCF90E8014EEAB0259
:10E50B0012EF590E0EAF060EA807E6FF12F007DC4E
:06E51B00F412F0F080BADA
:01E5210022D7
:04D50E008E308F319B
:10D51200853182853083E493FF54FC6063EF24FD00
:10D52200FE0531E53170020530C295F58285308302
:10D53200E493FC6402701F047B0112C86885318287
:10D54200F583E493FDAF0512F007DEF90531E5310D
:10D552007002053080248531828530837401AB04EA
:10D5620012C8680531E531AC307002053014F5821D
:10D572008C83E493FF12F007DEE912F0F002D51279
:01D582002286
:04C973008E2F8F3044
:10C9770012C861E49364FD700302CA1712C8B212A9
:10C98700C8BC7002052F12EFFF12C8BC7002052F3A
:10C9970012EFFF12C8A712C861E49364FC702674F3
:10C9A700029364FE701512C86174039314FC12C8D5
:10C9B700C3AF041CEF70EF7404802A12C86112C859
:10C9C700C37402802012C86174019364FE702174DD
:10C9D700029314FC12C861E493FF12F007AF041C22
:10C9E700EF70F174032530F530E4352FF52F800A09
:10C9F70012C8BC7002052F12EFFF12C861E493F44E
:10CA070070940530E5307002052F12F0F002C977F7
:01CA170022FC
:10F06600AE05C2957B01E4FD12EF5FAF0612F00715
:03F0760002F0F0B5
:10EAA300AE07AC03AA05C2957B017D0112EF5F128D
:10EAB300E9C9EF5A420412F0F0C295AF061D12EFF6
:09EAC3005FAF0412F00702F0F04D
:0CC070008E2A8F2B8C2C8D2D8A2E8B2F6E
:10C07C007480252DF52D7402352CF52C12C8B2E5E3
:10C08C002C540F44D0F531FF12F007E52DF531AFEC
:10C09C003112F00712C8A7E4F508F50AF50BC2181F
:10C0AC00F509E4F530AF2BAE2A12BC8978A612C183
:10C0BC003878A612C14578A712C13878A712C145A5
:10C0CC00EFC454F078A8F6AF2BAE2A12BC8978A82E
:10C0DC00E64FFFF618E6FEC454F0FDEF540F4DF595
:10C0EC003118E6FD540FFCEF54F04CF532EEC4540D
:10C0FC000FFFED54F04FF533E4FF74312FF8E6FEEB
:10C10C001312C853EE12C822D290D2940FBF03EA76
:10C11C000530E530C39409408CE52F152F700215BE
:0CC12C002E14452E600302C0AE02F0F09D
:10C13800EFC454F0F6AF2BAE2A12BC8922E64FF6B4
:08C14800AF2BAE2A12BC8922C4
:04BC89008E348F3531
:10BC8D00E4F536C219E508700FE535250BF582E5AB
:10BC9D003412C8887002050AE508D3940040E612F4
:10BCAD00C898301807201904D219800205363019AA
:10BCBD00E7E53614601714602514603314604114E1
:10BCCD006073240570D2C219E4F536FF2212BD69E6
:10BCDD00C219E4F5362018037F01227F0F2212BD11
:10BCED0069C219E4F5362018037F02227F0822125B
:10BCFD00BD71C219E4F5362018037F0C227F07228F
:10BD0D0012BD71C219E4F53630180C12BD79201828
:10BD1D00037F04227F092212BD7920180C12BD81E8
:10BD2D002018037F03227F0B2212BD812018037F71
:10BD3D000A227F052212BD89C219E4F53630180C8E
:10BD4D0012BD892018037F0E227F0D22AF35AE3430
:0BBD5D0012EF0A20180302BCA57F06AD
:10BD680022AF35AE3412EF0A22AF35AE3412EF0AE5
:10BD780022AF35AE3412EF0A22AF35AE3412EF0AD5
:09BD880022AF35AE3412EF0A229D
:10EF0A008F828E83E508700FE582250BF582E583F3
:0BEF1A0012C8887002050A12C8982275
:10E23400E52DA4FDACF0E531C4F8540FC868FFE542
:10E2440030C454F048FE1286E88F2EE4F530F531E0
:10E2540022540F4450F50F08E6252A22E52DA4FF89
:10E26400AEF0C3E5319FE5309E22750C06E4F50D52
:0EE27400750E9022FF7E007C001286D6EF22EF
:06944C008F298D2A8B2BF5
:10945200E478A6F608F6E52AFB7A0018A60208A622
:109462000374FB252BF52B7D0612E27824FAFFEE1E
:1094720034FFFEAD2C1286D68E308F3112E26EEBA7
:1094820078A726EA1836540F449012E259F510E5EF
:109492002EC454F0F511E4F5127F0C12E4D9750CC8
:1094A20005750D01750E92E52EC454F0F50F129656
:1094B20078E52A2405FDE52FC454F0F53875390204
:1094C2007B0CAF2912D82D12E26EF512F529E5298F
:1094D200C3952B4003029606E52A78A726FFE418D7
:1094E20036FE7C00EF2529FFEC3ECF2405CF340069
:1094F20012E25525292405F510E529600AE52B1409
:109502006529600302958DE5314530606F75F00382
:1095120012E2604010E52970047D1380027D1E8DE9
:1095220011C302959E75F00312E2347404D3952E92
:10953200400FE52970047F1080027F1B8F11029576
:10954200FC7408D3952E400FE52970047F11800228
:109552007F1C8F110295FC740CD3952E400FE529C8
:1095620070047F1280027F1D8F110295FCE5297025
:10957200047F1380027F1E8F110295FCE52970047F
:109582007F1080027F1B8F110295FCE53145306010
:109592006675F00612E260400F75111AE5319FF50B
:1095A20031E5309EF530805275F00612E23404D374
:1095B200952E400280417404D3952E4005751115F5
:1095C20080387406D3952E4005751116802C7409C7
:1095D200D3952E40057511178020740BD3952E401C
:1095E200057511188014740ED3952E400575111946
:1095F200800875111A80037511147F0C12E4D905C5
:10960200290294D0E52C75F00A84F52D75F00AA490
:10961200FFC3E52C9FF529E52D75F00A84F52E751B
:10962200F00AA4FFC3E52D9FF52D05297004E52E50
:109632006006E52D04FF80027F008F2DE52E600479
:1096420004FF80027F008F2E750C0512E271E52A5D
:1096520078A726E4183612E255129678750C06752C
:109662000D01750E92852E0F852D10852911E4F5B9
:06967200127F0C02E4D996
:0B967800F510E4F5117F0C12E4D9227C
:10E8100030091C300F1978A1E6FF6013F46010D2A4
:10E820001912EF25E4900F32F0900F3304F02220FC
:10E830000F0B900F337401F0900F32F022E4900F21
:08E8400033F0900F3204F022C6
:10DC8B0078CBE6605678C8E6604D78C9E6600D78CB
:10DC9B00CAE66003E4F622E478C9F622E478C8F613
:10DCAB00E67D2112E2782415FDE43EFCEF2433F5EA
:10DCBB0034E43EF5338C318D32E4F535F53675377A
:10DCCB000E7538FBF539753A01F53B7B1A7A017DF8
:0CDCDB0096FC7F0602B4BFE478CBF62272
:0300000002CF7AB2
:0CCF7A00787FE4F6D8FD7581D002CFC1AD
:10867E00BB010689828A83E0225002E722BBFE02FA
:09868E00E32289828A83E493222D
:10869700BB010CE58229F582E5833AF583E0225098
:1086A70006E92582F8E622BBFE06E92582F8E222E2
:0D86B700E58229F582E5833AF583E49322FC
:1086C400BB010689828A83F0225002F722BBFE0195
:0286D400F3228F
:1086D600EF8DF0A4A8F0CF8CF0A428CE8DF0A42EB8
:0286E600FE2272
:1086E800BC000BBE0029EF8DF084FFADF022E4CC76
:1086F800F875F008EF2FFFEE33FEEC33FCEE9DEC3F
:10870800984005FCEE9DFE0FD5F0E9E4CEFD22ED84
:10871800F8F5F0EE8420D21CFEADF075F008EF2FCE
:10872800FFED33FD4007985006D5F0F222C398FDBF
:058738000FD5F0EA225C
:10873D00E88FF0A4CC8BF0A42CFCE98EF0A42CFCDB
:10874D008AF0EDA42CFCEA8EF0A4CDA8F08BF0A459
:10875D002DCC3825F0FDE98FF0A42CCD35F0FCEBB8
:10876D008EF0A4FEA9F0EB8FF0A4CFC5F02ECD397D
:0F877D00FEE43CFCEAA42DCE35F0FDE43CFC22EA
:10878C0075F008758200EF2FFFEE33FECD33CDCCA4
:10879C0033CCC58233C5829BED9AEC99E582984027
:1087AC000CF582EE9BFEED9AFDEC99FC0FD5F0D604
:1087BC00E4CEFBE4CDFAE4CCF9A88222B800C1B92E
:1087CC000059BA002DEC8BF084CFCECDFCE5F0CB6C
:1087DC00F97818EF2FFFEE33FEED33FDEC33FCEBA5
:1087EC0033FB10D703994004EB99FB0FD8E5E4F960
:1087FC00FA227818EF2FFFEE33FEED33FDEC33FC4D
:10880C00C933C910D7059BE99A4007EC9BFCE99A40
:10881C00F90FD8E0E4C9FAE4CCFB2275F010EF2F85
:10882C00FFEE33FEED33FDCC33CCC833C810D70785
:10883C009BEC9AE899400AED9BFDEC9AFCE899F8C0
:0E884C000FD5F0DAE4CDFBE4CCFAE4C8F92253
:10885A00EB9FF5F0EA9E42F0E99D42F0E89C45F074
:01886A0022EB
:10886B00E8600FECC313FCED13FDEE13FEEF13FFEB
:03887B00D8F1220F
:10887E00E8600FEFC333FFEE33FEED33FDEC33FC58
:03888E00D8F122FC
:0C889100E6FC08E6FD08E6FE08E6FF2213
:0D889D00E6FB08E6F908E6FA08E6CBF8224B
:0C88AA00ECF608EDF608EEF608EFF622FA
:1088B600D083D082E493F608740193F60874029389
:0988C600F608740393F6740473C0
:0C88CF00A42582F582E5F03583F58322B4
:10CF860002D39FE493A3F8E493A34003F68001F24F
:10CF960008DFF48029E493A3F85407240CC8C333AC
:10CFA600C4540F4420C8834004F456800146F6DF7B
:10CFB600E4800B010204081020408090C225E47E24
:10CFC600019360BCA3FF543F30E509541FFEE49370
:10CFD600A360010ECF54C025E060A840B8E493A337
:10CFE600FAE493A3F8E493A3C8C582C8CAC583CA62
:10CFF600F0A3C8C582C8CAC583CADFE9DEE780BE1A
:01C2F5000048
:00000001FF
